:020000040000FA
:040800004DEF0BF0BD
:1008100003B276EF05F0F2B494EF05F09EB09CEFD2
:1008200005F09EB2A4EF05F0F2A81AEF04F0F2B2C0
:1008300025EF04F0F2A620EF04F0F2B022EF04F06E
:10084000FCEF0AF0F296F290FF00CD90F2929EA09B
:100850002FEF04F00101533F2FEF04F0542BAEC1F2
:10086000B2F1AFC1B3F1B0C1B4F1B1C1B5F1AAC138
:10087000AEF1ABC1AFF1ACC1B0F1ADC1B1F1A6C148
:10088000AAF1A7C1ABF1A8C1ACF1A9C1ADF1A2C158
:10089000A6F1A3C1A7F1A4C1A8F1A5C1A9F19EC168
:1008A000A2F19FC1A3F1A0C1A4F1A1C1A5F19AC178
:1008B0009EF19BC19FF19CC1A0F19DC1A1F196C188
:1008C0009AF197C19BF198C19CF199C19DF1CECF4E
:1008D00096F1CFCF97F153C198F154C199F1CF6AF6
:1008E000CE6A0101536B546B9E90CD800FBC0F8E6E
:1008F0000FBA7EEF04F00F8AFCEF0AF00F8C0FBEE8
:10090000BAEF04F096C19AF197C19BF198C19CF19E
:1009100099C19DF19AC19EF19BC19FF19CC1A0F12B
:100920009DC1A1F19EC1A2F19FC1A3F1A0C1A4F1FB
:10093000A1C1A5F1A2C1A6F1A3C1A7F1A4C1A8F1CB
:10094000A5C1A9F1A6C1AAF1A7C1ABF1A8C1ACF19B
:10095000A9C1ADF1AAC1AEF1ABC1AFF1ACC1B0F16B
:10096000ADC1B1F1AEC1B2F1AFC1B3F1B0C1B4F13B
:10097000B1C1B5F101015E6B5F6B606B616B96514C
:100980005E2797515F2398516023995161239A51B3
:100990005E279B515F239C5160239D5161239E5193
:1009A0005E279F515F23A0516023A1516123A25173
:1009B0005E27A3515F23A4516023A5516123A65153
:1009C0005E27A7515F23A8516023A9516123AA5133
:1009D0005E27AB515F23AC516023AD516123AE5113
:1009E0005E27AF515F23B0516023B1516123B251F3
:1009F0005E27B3515F23B4516023B5516123D89072
:100A00000101613360335F335E33D890010161339C
:100A100060335F335E33D8900101613360335F33FD
:100A20005E3300C10CF101C10DF102C10EF103C131
:100A30000FF104C110F105C111F106C112F107C196
:100A400013F108C114F109C115F10AC116F10BC166
:100A500017F134C135F111B839EF05F00101620E1B
:100A6000046F010E056F000E066F000E076F42EF58
:100A700005F00101A70E046F020E056F000E066F50
:100A8000000E076F5EC100F15FC101F160C102F1AC
:100A900061C103F1C2EC2AF003BF04D018BE02D03A
:100AA00018A0108C11A05AEF05F010BA5AEF05F0FB
:100AB0000F80108A0CC100F10DC101F10EC102F1CD
:100AC0000FC103F110C104F111C105F112C106F10A
:100AD00013C107F114C108F115C109F116C10AF1DA
:100AE00017C10BF135C134F1FCEF0AF00392ABB240
:100AF000AB98AB88030103EE00F080517F0BE92631
:100B000004C0EFFF802B8151805D700BD8A48B82D5
:100B100000008051815D700BD8A48B9281518019A7
:100B2000D8B40790FCEF0AF0F2940101453FFCEFC6
:100B30000AF0462BFCEF0AF09E900101533FFCEFB8
:100B40000AF0542BFCEF0AF09E9211B821EF08F046
:100B5000040066A1ACEF05F08BB4B6EF05F010AC65
:100B6000B6EF05F08B84109CB7EF05F08B94077CF3
:100B700007ACD2EF05F0C274C2B4CCEF05F0C3CF1E
:100B8000B7F5C4CFB8F50501D890B833B733D890CE
:100B9000B833B733D3EF05F0C3CF55F1C4CF56F117
:100BA000D3EF05F0C28207B440EF06F047C14BF126
:100BB00048C14CF149C14DF14AC14EF15EC162F1EB
:100BC0005FC163F160C164F161C165F196C1B6F1C5
:100BD00097C1B7F198C1B8F199C1B9F19AC1BAF109
:100BE0009BC1BBF19CC1BCF19DC1BDF19EC1BEF1D9
:100BF0009FC1BFF1A0C1C0F1A1C1C1F1A2C1C2F1A9
:100C0000A3C1C3F1A4C1C4F1A5C1C5F1A6C1C6F178
:100C1000A7C1C7F1A8C1C8F1A9C1C9F1AAC1CAF148
:100C2000ABC1CBF1ACC1CCF1ADC1CDF1AEC1CEF118
:100C3000AFC1CFF1B0C1D0F1B1C1D1F1B2C1D2F1E8
:100C4000B3C1D3F1B4C1D4F1B5C1D5F1B7C5B9F5CC
:100C5000B8C5BAF5B9C5BBF5BAC5BCF50101555162
:100C60005B2756515C23E86A5D230E2E40EF06F0A9
:100C70005CC157F15DC158F15B6B5C6B5D6B078EBE
:100C80000201002FFCEF0AF03C0E006F1950E00B40
:100C9000E00AE866128817BE02D017B4108E00C1B1
:100CA0000CF101C10DF102C10EF103C10FF104C13C
:100CB00010F105C111F106C112F107C113F108C10C
:100CC00014F109C115F10AC116F10BC117F134C1B4
:100CD00035F105012F51000AD8B41AEF07F00501CC
:100CE0002F51010AD8B4A4EF06F005012F51020AD2
:100CF000D8B4E5EF06F005012F51030AD8B4E5EFAB
:100D000006F005012F51040AD8B4E5EF06F00501FD
:100D10002F51050AD8B4E5EF06F005012F51060A58
:100D2000D8B4E5EF06F005012F51070AD8B4E5EF76
:100D300006F005012F51320AD8B4A2EF06F02F6B4E
:100D40001AEF07F01AEF07F005015767AFEF06F04B
:100D50005867AFEF06F05967AFEF06F05A67B3EF89
:100D600006F01AEF07F05BC500F15CC501F15DC547
:100D700002F15EC503F10101010E046F000E056F63
:100D8000000E066F000E076FC2EC2AF000C15BF583
:100D900001C15CF502C15DF503C15EF50067D8EFE6
:100DA00006F00167D8EF06F00267D8EF06F0036798
:100DB0001AEF07F057C55BF558C55CF559C55DF5E9
:100DC0005AC55EF50F881AEF07F005013067EBEFA3
:100DD00006F01AEF07F00FBE00EF07F010A005EFC6
:100DE00007F001014767FCEF06F04867FCEF06F0EB
:100DF0004967FCEF06F04A6700EF07F005EF07F0E0
:100E000007AE05EF07F017EF07F00501312F1AEFD6
:100E100007F03C0E316F302F1AEF07F00101000E82
:100E2000626FE00E636FA50E646F010E656F0501C2
:100E3000306B0F880501666B37B720EF07F06681CE
:100E40000CC100F10DC101F10EC102F10FC103F19E
:100E500010C104F111C105F112C106F113C107F16E
:100E600014C108F115C109F116C10AF117C10BF13E
:100E700035C134F100C10CF101C10DF102C10EF117
:100E800003C10FF104C110F105C111F106C112F146
:100E900007C113F108C114F109C115F10AC116F116
:100EA0000BC117F134C135F101018A675FEF07F01B
:100EB0008B675FEF07F08C675FEF07F08D6763EF7D
:100EC00007F093EF07F08EC100F18FC101F190C1DF
:100ED00002F191C103F10101010E046F000E056FD3
:100EE000000E066F000E076FC2EC2AF000C18EF1F3
:100EF00001C18FF102C190F103C191F1006788EF48
:100F000007F0016788EF07F0026788EF07F00367D3
:100F100093EF07F08AC18EF18BC18FF18CC190F1F4
:100F20008DC191F10F80D57ED5BE6DD0D6CF47F162
:100F3000D7CF48F145C149F1E86AE8CF4AF118BE78
:100F400002D018A0108C109047C100F148C101F1E7
:100F500049C102F14AC103F101010A0E046F000EFA
:100F6000056F000E066F000E076FC2EC2AF003AF8C
:100F70001080010154A7C9EF07F00F9A0F9C0F9E34
:100F80000101000E5E6F600E5F6F3D0E606F080E18
:100F9000616F010147BFD9EF07F04867D9EF07F04C
:100FA0004967D9EF07F04A67D9EF07F0F288FEEFFB
:100FB00007F0F2985E6B5F6B606B616B966B976B83
:100FC000986B996B9A6B9B6B9C6B9D6B9E6B9F6BED
:100FD000A06BA16BA26BA36BA46BA56BA66BA76B9D
:100FE000A86BA96BAA6BAB6BAC6BAD6BAE6BAF6B4D
:100FF000B06BB16BB26BB36BB46BB56BD76AD66ABF
:101000000101456B466B0CC100F10DC101F10EC130
:1010100002F10FC103F110C104F111C105F112C1B8
:1010200006F113C107F114C108F115C109F116C188
:101030000AF117C10BF135C134F1FCEF0AF0FCEFF6
:101040000AF00201002F65EF0AF0D59ED6CF47F1D6
:10105000D7CF48F145C149F1E86AE8CF4AF1D76AEC
:10106000D66A0101456B466BD58E1950E00BE00A3C
:10107000E866128817BE02D017B4108E16AE1B8C0D
:1010800000C10CF101C10DF102C10EF103C10FF15C
:1010900004C110F105C111F106C112F107C113F12C
:1010A00008C114F109C115F10AC116F10BC117F1FC
:1010B00034C135F10FA0109A11B86AEF08F00101A0
:1010C000620E046F010E056F000E066F000E076FB3
:1010D00073EF08F00101A70E046F020E056F000EFA
:1010E000066F000E076F47C100F148C101F149C109
:1010F00002F14AC103F1C2EC2AF003BF86EF08F007
:1011000018BE02D018A0108C11B00F800CC100F1D5
:101110000DC101F10EC102F10FC103F110C104F1C3
:1011200011C105F112C106F113C107F114C108F193
:1011300015C109F116C10AF117C10BF135C134F11E
:1011400002013C0E006F00C10CF101C10DF102C1A2
:101150000EF103C10FF104C110F105C111F106C177
:1011600012F107C113F108C114F109C115F10AC147
:1011700016F10BC117F134C135F105012F51000AE9
:10118000D8B46EEF09F005012F51010AD8B4F8EF79
:1011900008F005012F51020AD8B439EF09F0050112
:1011A0002F51030AD8B439EF09F005012F51040A71
:1011B000D8B439EF09F005012F51050AD8B439EF39
:1011C00009F005012F51060AD8B439EF09F00501DD
:1011D0002F51070AD8B439EF09F005012F51320A0F
:1011E000D8B4F6EF08F02F6B6EEF09F06EEF09F050
:1011F0000501576703EF09F0586703EF09F05967D6
:1012000003EF09F05A6707EF09F06EEF09F05BC5CD
:1012100000F15CC501F15DC502F15EC503F101019C
:10122000010E046F000E056F000E066F000E076FB3
:10123000C2EC2AF000C15BF501C15CF502C15DF5AD
:1012400003C15EF500672CEF09F001672CEF09F090
:1012500002672CEF09F003676EEF09F057C55BF5E5
:1012600058C55CF559C55DF55AC55EF50F886EEF3A
:1012700009F0050130673FEF09F06EEF09F00FBE8E
:1012800054EF09F010A059EF09F00101476750EF42
:1012900009F0486750EF09F0496750EF09F04A67D5
:1012A00054EF09F059EF09F007AE59EF09F06BEF71
:1012B00009F00501312F6EEF09F03C0E316F302F30
:1012C0006EEF09F00101000E626FE00E636FA50E74
:1012D000646F010E656F0501306B0F880501666B49
:1012E00037B774EF09F066810CC100F10DC101F14F
:1012F0000EC102F10FC103F110C104F111C105F1DA
:1013000012C106F113C107F114C108F115C109F1A9
:1013100016C10AF117C10BF135C134F100C10CF14E
:1013200001C10DF102C10EF103C10FF104C110F1B1
:1013300005C111F106C112F107C113F108C114F181
:1013400009C115F10AC116F10BC117F134C135F10C
:1013500001018A67B3EF09F08B67B3EF09F08C677F
:10136000B3EF09F08D67B7EF09F0E7EF09F08EC131
:1013700000F18FC101F190C102F191C103F10101AE
:10138000010E046F000E056F000E066F000E076F52
:10139000C2EC2AF000C18EF101C18FF102C190F1BF
:1013A00003C191F10067DCEF09F00167DCEF09F0A0
:1013B0000267DCEF09F00367E7EF09F08AC18EF1FD
:1013C0008BC18FF18CC190F18DC191F10F80109084
:1013D00047C100F148C101F149C102F14AC103F11D
:1013E00001010A0E046F000E056F000E066F000E5D
:1013F000076FC2EC2AF003AF1080010154A70DEF74
:101400000AF00F9A0F9C0F9E0101000E5E6F600E96
:101410005F6F3D0E606F080E616F47C100F148C1FC
:1014200001F149C102F14AC103F10101140E046F37
:10143000050E056F000E066F000E076FC2EC2AF056
:1014400003AF26EF0AF0F2884BEF0AF0F2985E6BDA
:101450005F6B606B616B966B976B986B996B9A6B1C
:101460009B6B9C6B9D6B9E6B9F6BA06BA16BA26B30
:10147000A36BA46BA56BA66BA76BA86BA96BAA6BE0
:10148000AB6BAC6BAD6BAE6BAF6BB06BB16BB26B90
:10149000B36BB46BB56B0CC100F10DC101F10EC1A2
:1014A00002F10FC103F110C104F111C105F112C124
:1014B00006F113C107F114C108F115C109F116C1F4
:1014C0000AF117C10BF135C134F104008BB470EF90
:1014D0000AF010AC70EF0AF08B84109C71EF0AF0E8
:1014E0008B94077C07AC8CEF0AF0C274C2B486EF11
:1014F0000AF0C3CFB7F5C4CFB8F50501D890B8331B
:10150000B733D890B833B7338DEF0AF0C3CF55F166
:10151000C4CF56F18DEF0AF0C28207B4FAEF0AF099
:1015200047C14BF148C14CF149C14DF14AC14EF19F
:101530005EC162F15FC163F160C164F161C165F1D7
:1015400096C1B6F197C1B7F198C1B8F199C1B9F197
:101550009AC1BAF19BC1BBF19CC1BCF19DC1BDF167
:101560009EC1BEF19FC1BFF1A0C1C0F1A1C1C1F137
:10157000A2C1C2F1A3C1C3F1A4C1C4F1A5C1C5F107
:10158000A6C1C6F1A7C1C7F1A8C1C8F1A9C1C9F1D7
:10159000AAC1CAF1ABC1CBF1ACC1CCF1ADC1CDF1A7
:1015A000AEC1CEF1AFC1CFF1B0C1D0F1B1C1D1F177
:1015B000B2C1D2F1B3C1D3F1B4C1D4F1B5C1D5F147
:1015C000B7C5B9F5B8C5BAF5B9C5BBF5BAC5BCF567
:1015D000010155515B2756515C23E86A5D230E2EAD
:1015E000FAEF0AF05CC157F15DC158F15B6B5C6BBF
:1015F0005D6B078EFCEF0AF002C0E0FF005001C0F7
:10160000D8FF1000A6B202EF0BF00CC0A9FF0BC070
:10161000A8FFA69EA69CA684F29E550EA76EAA0EB3
:10162000A76EA682F28EA694A6B214EF0BF00C2A37
:101630001200A96EA69EA69CA680A8500C2A120095
:1016400004012C0E826F5EEC0EF0BDEC2BF00C5002
:1016500019EC0BF0E8CF00F10C5019EC0BF0E8CFCF
:1016600001F101AF39EF0BF00101FF0E026FFF0E28
:10167000036F60EC2BF0296745EF0BF00401200E9F
:10168000826F5EEC0EF04AEF0BF004012D0E826FBC
:101690005EEC0EF08AEC29F01200076A0F6A106AFD
:1016A000116A126A0F010D0EC16E860EC06E030E16
:1016B000C26E0F01680E896E130E926E080E8A6E4E
:1016C000F30E936E8B6A900E946EC80E19EC0BF0AD
:1016D000E8CFE8FF1098E8A0108810A805D00E0EFB
:1016E000216E8E0E226E04D00F0E216E8F0E226E92
:1016F0003CEC2CF0F18EF19EFC0E19EC0BF0E8CFD7
:101700000BF00BA011800BA211820BA411840BA86B
:101710001188C90E19EC0BF0E8CF16F0CA0E19ECBF
:101720000BF0E8CF17F0CB0E19EC0BF0E8CF18F068
:10173000CC0E19EC0BF0E8CF19F01B6A1C6A0E6A8C
:1017400001015B6B5C6B5D6B576B586BF29A01012F
:10175000476B486B496B4A6B4B6B4C6B4D6B4E6BDD
:101760004F6B506B516B526B456B466BD76AD66AA9
:101770000F01280ED56EF28A9D90B00ECD6E01013C
:101780005E6B5F6B606B616B626B636B646B656BF5
:10179000666B676B686B696B536B546BCF6ACE6A11
:1017A0000F9A0F9C0F9E9D80760ECA6E9D8202013D
:1017B0003C0E006FCC6A160E19EC0BF0E8CF00F16E
:1017C000170E19EC0BF0E8CF01F1180E19EC0BF025
:1017D000E8CF02F1190E19EC0BF0E8CF03F101018B
:1017E00003AF0DEF0CF0BDEC2BF0160E0C6E00C12C
:1017F0000BF002EC0BF0170E0C6E01C10BF002ECBB
:101800000BF0180E0C6E02C10BF002EC0BF0190E6F
:101810000C6E03C10BF002EC0BF000C18AF101C1A8
:101820008BF102C18CF103C18DF100C18EF101C1B8
:101830008FF102C190F103C191F11A0E19EC0BF076
:10184000E8CF00F11B0E19EC0BF0E8CF01F11C0EF4
:1018500019EC0BF0E8CF02F11D0E19EC0BF0E8CFFC
:1018600003F1010103AF63EF0CF0BDEC2BF01A0E96
:101870000C6E00C10BF002EC0BF01B0E0C6E01C1E4
:101880000BF002EC0BF01C0E0C6E02C10BF002EC24
:101890000BF01D0E0C6E03C10BF002EC0BF01A0ED8
:1018A00019EC0BF0E8CF00F11B0E19EC0BF0E8CFB0
:1018B00001F11C0E19EC0BF0E8CF02F11D0E19EC32
:1018C0000BF0E8CF03F100C192F101C193F102C125
:1018D00094F103C195F1240EAC6E900EAB6E240E04
:1018E000AC6E080EB86E000EB06E1F0EAF6E040127
:1018F000806B816B0F01900EAB6E0F019D8A03010F
:10190000806B816BC26B8B92C4EC30F0C4EC30F016
:1019100020EC32F0A3EC2EF0200E19EC0BF0E8CF07
:101920002FF505012F51FF0AD8A49EEF0CF02F6B65
:10193000200E0C6E2FC50BF002EC0BF00501010E12
:10194000306F3C0E316F250E19EC0BF0E8CF00F133
:10195000260E19EC0BF0E8CF01F1270E19EC0BF075
:10196000E8CF02F1280E19EC0BF0E8CF03F10101EA
:1019700003AFD5EF0CF0BDEC2BF0250E0C6E00C1C3
:101980000BF002EC0BF0260E0C6E01C10BF002EC1A
:101990000BF0270E0C6E02C10BF002EC0BF0280EC0
:1019A0000C6E03C10BF002EC0BF000C157F501C146
:1019B00058F502C159F503C15AF500C15BF501C1E3
:1019C0005CF502C15DF503C15EF5290E19EC0BF063
:1019D000E8CF5FF5050160515F5DD8A05FC560F598
:1019E00005012F51020A0EE181B802EF0DF0050149
:1019F000602FFFEF0CF05FC560F502EF0DF081BACC
:101A00005FEF32F0210E19EC0BF0E8CF00F1220E5F
:101A100019EC0BF0E8CF01F1230E19EC0BF0E8CF35
:101A200002F1240E19EC0BF0E8CF03F1010103AF32
:101A300048EF0DF0BDEC2BF0210E0C6E00C10BF049
:101A400002EC0BF0220E0C6E01C10BF002EC0BF05D
:101A5000230E0C6E02C10BF002EC0BF0240E0C6E88
:101A600003C10BF002EC0BF0210E19EC0BF0E8CFE8
:101A700000F1220E19EC0BF0E8CF01F1230E19EC66
:101A80000BF0E8CF02F1240E19EC0BF0E8CF03F1D4
:101A900000C161F501C162F502C163F503C164F5DE
:101AA000EBEC2DF0EDEC2CF045EC2CF005012F517A
:101AB000030A12E005012F51040A1DE005012F5110
:101AC000050A24E005012F51060A32E005012F51D5
:101AD000070A38E0ABEF0DF0B0C500F101010F0EC1
:101AE000001701010051000A36E001010051050A0A
:101AF00032E0A8EF0DF0B0C500F101010F0E0017A4
:101B000001010051000A27E0A8EF0DF00501B051D6
:101B1000000A21E00501B051150A1DE00501B05190
:101B2000300A19E00501B051450A15E0A8EF0DF0A3
:101B30000501B051000A0FE00501B051300A0BE079
:101B4000A8EF0DF00501B051000A05E0A8EF0DF077
:101B500081BA5FEF32F007900001F28EF28C12BE74
:101B600072EF17F007B00CEF28F00FB0A8EF21F0DC
:101B700010BEA8EF21F012B8A8EF21F00FB845EF82
:101B80001BF00301805181197F0BD8B40CEF28F0B2
:101B900013EE00F081517F0BE126812BE7CFE8FFA8
:101BA000E00BD8B40CEF28F023EE82F0C2513F0BCB
:101BB000D926E7CFDFFFC22BDF50780AD8A40CEF7D
:101BC00028F007808EC100F18FC101F190C102F1B0
:101BD00091C103F10101040E046F000E056F000EA8
:101BE000066F000E076FC2EC2AF000AF01EF0EF097
:101BF0000101030E8E6F000E8F6F000E906F000EAE
:101C0000916F03018251720AD8B48DEF21F0825195
:101C1000520AD8B48DEF21F08251750AD8B48DEFF5
:101C200021F08251630AD8B4C6EF24F08251690AC8
:101C3000D8B43CEF1EF082517A0AD8B44FEF1FF0AF
:101C40008251490AD8B4DBEF1DF08251500AD8B452
:101C5000F9EF1CF08251700AD8B43CEF1DF08251AC
:101C6000540AD8B467EF1DF08251740AD8B4ADEFAE
:101C70001DF08251410AD8B472EF0EF082516D0A04
:101C8000D8B47CEF12F082514D0AD8B495EF12F01F
:101C90008251730AD8B4BDEF20F08251530AD8B4F0
:101CA00022EF21F082514C0AD8B424EF13F0825174
:101CB000590AD8B4CDEF11F0FDEF24F0040114EE71
:101CC00000F080517F0BE12682C4E7FF802B1200D9
:101CD00004010D0E826F5EEC0EF00A0E826F5EEC58
:101CE0000EF012000401410E826F5EEC0EF0030153
:101CF0008351310AD8B4EDEF10F003018351320A59
:101D0000D8B41DEF10F003018351330AD8B4A6EF05
:101D10000FF003018351340AD8B496EF0EF004019A
:101D20003F0E826F5EEC0EF0FBEF24F0CC0E19EC50
:101D30000BF0E8CF0BF004012C0E826F5EEC0EF07E
:101D400003018451310AD8B4BAEF0EF00301845173
:101D5000300AD8B4BCEF0EF0030184514D0AD8B458
:101D6000C6EF0EF003018451540AD8B4CDEF0EF043
:101D7000E4EF0EF08A8401D08A940BAE04D00BAC51
:101D800002D00BBA21D0E00E0B1218D01F0E0B168A
:101D90008539E844E00B0B1211D0E00E0B16FEEC77
:101DA0002BF085C332F186C333F10101296B0BECB3
:101DB0002CF082EC2BF000511F0B0B12CC0E0C6E92
:101DC0000BC00BF002EC0BF00401340E826F5EECE2
:101DD0000EF004012C0E826F5EEC0EF0CC0E19ECAE
:101DE0000BF0E8CF19F08AB406D00401300E826FF0
:101DF0005EEC0EF005D00401310E826F5EEC0EF049
:101E000004012C0E826F5EEC0EF01938E840070BCF
:101E1000E8CF82F40401300E82275EEC0EF004015C
:101E20002C0E826F5EEC0EF0BDEC2BF019501F0BE8
:101E3000E8CF00F160EC2BF032C182F40401300EE7
:101E400082275EEC0EF033C182F40401300E82274B
:101E50005EEC0EF004012C0E826F5EEC0EF0BDEC19
:101E60002BF02CC000F100AF0BD0FF0E016FFF0E66
:101E7000026FFF0E036F04012D0E826F5EEC0EF0F9
:101E800060EC2BF031C182F40401300E82275EEC4D
:101E90000EF032C182F40401300E82275EEC0EF0A7
:101EA00033C182F40401300E82275EEC0EF004018F
:101EB0002C0E826F5EEC0EF0BDEC2BF02BC000F10F
:101EC00060EC2BF031C182F40401300E82275EEC0D
:101ED0000EF032C182F40401300E82275EEC0EF067
:101EE00033C182F40401300E82275EEC0EF004014F
:101EF0002C0E826F5EEC0EF0BDEC2BF02DC000F1CD
:101F000000AF0BD0FF0E016FFF0E026FFF0E036FCD
:101F100004012D0E826F5EEC0EF060EC2BF031C1EF
:101F200082F40401300E82275EEC0EF032C182F49E
:101F30000401300E82275EEC0EF033C182F40401FE
:101F4000300E82275EEC0EF0FBEF24F0CB0E19EC86
:101F50000BF0E8CF0BF004012C0E826F5EEC0EF05C
:101F600003018451450AD8B4CAEF0FF0030184512C
:101F7000440AD8B4CDEF0FF003018451300AD8B42D
:101F8000D0EF0FF003018451310AD8B4D4EF0FF031
:101F9000DFEF0FF00B9ED9EF0FF00B8ED9EF0FF0A4
:101FA000FC0E0B16D9EF0FF0FC0E0B160B80D9EFC1
:101FB0000FF0CB0E0C6E0BC00BF002EC0BF004011B
:101FC000330E826F5EEC0EF004012C0E826F5EEC1D
:101FD0000EF0CB0E19EC0BF0E8CF18F018BEF8EFAE
:101FE0000FF00401450E826F5EEC0EF0FDEF0FF076
:101FF0000401440E826F5EEC0EF004012C0E826F21
:102000005EEC0EF00401300E826F5EEC0EF0040107
:102010002C0E826F5EEC0EF018B016EF10F004017B
:10202000300E826F5EEC0EF01BEF10F00401310EEB
:10203000826F5EEC0EF0FBEF24F0CA0E19EC0BF091
:10204000E8CF0BF004012C0E826F5EEC0EF0030162
:102050008451450AD8B459EF10F003018451440A61
:10206000D8B45CEF10F0030184514D0AD8B465EF89
:1020700010F003018451410AD8B45FEF10F003015E
:102080008451460AD8B462EF10F003018451560A15
:10209000D8B46DEF10F003018451500AD8B478EF32
:1020A00010F003018451520AD8B47BEF10F084EF92
:1020B00010F00B9E7EEF10F00B8E7EEF10F00B9C5D
:1020C0007EEF10F00B8C7EEF10F0FC0E0B1685C32C
:1020D000E8FF030B0B127EEF10F0C70E0B1685C343
:1020E000E8FF070BE846E846E8460B127EEF10F0E3
:1020F0000B847EEF10F00B947EEF10F0CA0E0C6E86
:102100000BC00BF002EC0BF0CA0E19EC0BF0E8CF91
:1021100017F00401320E826F5EEC0EF004012C0EFB
:10212000826F5EEC0EF017BE9DEF10F00401450EBD
:10213000826F5EEC0EF0A2EF10F00401440E826F8D
:102140005EEC0EF004012C0E826F5EEC0EF017C0F8
:10215000E8FF030BE8CF82F40401300E82275EEC27
:102160000EF004012C0E826F5EEC0EF017BCC0EF77
:1021700010F00401410E826F5EEC0EF0C5EF10F01E
:102180000401460E826F5EEC0EF004012C0E826F8D
:102190005EEC0EF017C0E8FF380BE842E842E84278
:1021A000E8CF82F40401300E82275EEC0EF00401C9
:1021B0002C0E826F5EEC0EF017B4E6EF10F0040107
:1021C000520E826F5EEC0EF0EBEF10F00401500E39
:1021D000826F5EEC0EF0FBEF24F0C90E19EC0BF0F1
:1021E000E8CF0BF004012C0E826F5EEC0EF00301C1
:1021F0008451450AD8B40BEF11F003018451440A0D
:10220000D8B40EEF11F0030184514D0AD8B411EF88
:1022100011F01FEF11F00B9E19EF11F00B8E19EF5B
:1022200011F0F80E0B1685C3E8FF070B0B1219EF20
:1022300011F0C90E0C6E0BC00BF002EC0BF0040198
:10224000310E826F5EEC0EF004012C0E826F5EEC9C
:102250000EF0C90E19EC0BF0E8CF16F016BE06D042
:102260000401450E826F5EEC0EF005D00401440EB1
:10227000826F5EEC0EF004012C0E826F5EEC0EF0AD
:1022800016C0E8FF070BE8CF82F40401300E822766
:102290005EEC0EF004012C0E826F5EEC0EF00780F7
:1022A000BDEC2BF027C0E8FF003B00430043030BCD
:1022B00060EC2BF033C182F40401300E82275EEC17
:1022C0000EF004012C0E826F5EEC0EF0BDEC2BF0D4
:1022D00027C001F1019F019D28C000F1010160ECC0
:1022E0002BF02FC182F40401300E82275EEC0EF039
:1022F00030C182F40401300E82275EEC0EF031C151
:1023000082F40401300E82275EEC0EF032C182F4BA
:102310000401300E82275EEC0EF033C182F404011A
:10232000300E82275EEC0EF004012C0E826F5EEC04
:102330000EF0BDEC2BF029C001F12AC000F1D890BD
:1023400001330033D89001330033010160EC2BF0EE
:102350002FC182F40401300E82275EEC0EF030C1F2
:1023600082F40401300E82275EEC0EF031C182F45B
:102370000401300E82275EEC0EF032C182F40401BB
:10238000300E82275EEC0EF033C182F40401300E71
:1023900082275EEC0EF0FBEF24F0FC0E19EC0BF044
:1023A000E8CF0BF003018351520AD8B404EF12F0C6
:1023B00003018351720AD8B407EF12F0030183516D
:1023C000500AD8B40AEF12F003018351700AD8B44E
:1023D0000DEF12F003018351550AD8B410EF12F03B
:1023E00003018351750AD8B413EF12F0030183512E
:1023F000430AD8B41CEF12F003018351630AD8B426
:102400001FEF12F028EF12F00B9022EF12F00B806A
:1024100022EF12F00B9222EF12F00B8222EF12F059
:102420000B9422EF12F00B8422EF12F00B9622EFA6
:1024300012F00B8622EF12F00B9822EF12F00B88AD
:1024400022EF12F0FC0E0C6E0BC00BF002EC0BF046
:102450000401590E826F5EEC0EF0119011921194EE
:102460001198FC0E19EC0BF0E8CF0BF00BA01180CB
:102470000BA211820BA411840BA8118811A048EFA4
:1024800012F00401520E826F5EEC0EF04DEF12F06E
:102490000401720E826F5EEC0EF011A857EF12F07D
:1024A0000401430E826F5EEC0EF05CEF12F004014B
:1024B000630E826F5EEC0EF011A266EF12F0040163
:1024C000500E826F5EEC0EF06BEF12F00401700E96
:1024D000826F5EEC0EF011A475EF12F00401550E40
:1024E000826F5EEC0EF07AEF12F00401750E826FCF
:1024F0005EEC0EF0FBEF24F004016D0E826F5EECDB
:102500000EF003018351300AD8B4D4EF12F0030166
:102510008351310AD8B4E7EF12F003018351320A34
:10252000D8B4FAEF12F0FDEF24F004014D0E826FE3
:102530005EEC0EF0FEEC2BF084C331F185C332F17A
:1025400086C333F10101296B0BEC2CF082EC2BF0EC
:1025500003018351300AD8B4BCEF12F00301835158
:10256000310AD8B4C4EF12F003018351320AD8B44F
:10257000CCEF12F0FDEF24F0FD0E0C6E00C10BF05D
:1025800002EC0BF0D4EF12F0FE0E0C6E00C10BF05B
:1025900002EC0BF0E7EF12F0FF0E0C6E00C10BF037
:1025A00002EC0BF0FAEF12F00401300E826F5EECD9
:1025B0000EF004012C0E826F5EEC0EF0BDEC2BF0E1
:1025C000FD0E19EC0BF0E8CF00F10BEF13F0040156
:1025D000310E826F5EEC0EF004012C0E826F5EEC09
:1025E0000EF0BDEC2BF0FE0E19EC0BF0E8CF00F175
:1025F0000BEF13F00401320E826F5EEC0EF0BDECB7
:102600002BF004012C0E826F5EEC0EF0FF0E19EC25
:102610000BF0E8CF00F160EC2BF031C182F4040143
:10262000300E82275EEC0EF032C182F40401300ECF
:1026300082275EEC0EF033C182F40401300E822753
:102640005EEC0EF0FBEF24F003018351300AD8B4A6
:102650001EEF18F003018351310AD8B44BEF19F083
:1026600003018351320AD8B4B9EF19F00301835141
:10267000330AD8B4C9EF19F003018351340AD8B42E
:10268000D9EF19F003018351350AD8B44AEF1BF092
:1026900003018351360AD8B478EF1BF0030183514C
:1026A000370AD8B4F7EF15F003018351380AD8B4CC
:1026B00095EF16F003018351460AD8B49EEF1AF045
:1026C000030183514D0AD8B470EF14F00301835114
:1026D0006D0AD8B48AEF14F0030183515A0AD8B4B2
:1026E000C5EF18F003018351490AD8B478EF1CF004
:1026F00003018351500AD8B4AAEF1BF003018351A0
:10270000540AD8B423EF1CF003018351630AD8B4F0
:10271000AAEF14F003018351430AD8B4A2EF15F0D5
:1027200003018351730AD8B4A8EF14F00301835155
:10273000610AD8B4BDEF13F003018351650AD8B420
:102740006EEF18F003018351450AD8B47CEF18F0FE
:1027500003018351620AD8B48AEF18F00301835150
:10276000420AD8B498EF18F003018351760AD8B41E
:10277000A6EF18F0D8A4FDEF24F004014C0E826FF0
:102780005EEC0EF00401610E826F5EEC0EF0EDEC7B
:102790002CF004012C0E826F5EEC0EF0BDEC2BF0E1
:1027A000AFC500F1010160EC2BF031C182F40401EE
:1027B000300E82275EEC0EF032C182F40401300E3E
:1027C00082275EEC0EF033C182F40401300E8227C2
:1027D0005EEC0EF004012C0E826F5EEC0EF0BDEC90
:1027E0002BF0B0C500F1010160EC2BF031C182F497
:1027F0000401300E82275EEC0EF032C182F4040137
:10280000300E82275EEC0EF033C182F40401300EEC
:1028100082275EEC0EF004012C0E826F5EEC0EF04F
:10282000BDEC2BF0B1C500F1010160EC2BF031C122
:1028300082F40401300E82275EEC0EF032C182F485
:102840000401300E82275EEC0EF033C182F40401E5
:10285000300E82275EEC0EF004012C0E826F5EECCF
:102860000EF0BDEC2BF0B2C500F1010160EC2BF0D5
:1028700031C182F40401300E82275EEC0EF032C1C9
:1028800082F40401300E82275EEC0EF033C182F434
:102890000401300E82275EEC0EF004012C0E826FD4
:1028A0005EEC0EF0BDEC2BF0B6C500F1010160EC62
:1028B0002BF031C182F40401300E82275EEC0EF061
:1028C00032C182F40401300E82275EEC0EF033C177
:1028D00082F40401300E82275EEC0EF0A6EF1BF0AE
:1028E000FEEC2BF084C333F10BEC2CF082EC2BF0DC
:1028F000200E0C6E00C10BF002EC0BF000C12FF5A6
:1029000005012F51000A06E005012F51010A02E0DE
:1029100087EC2DF004014C0E826F5EEC0EF004018A
:102920004D0E826F5EEC0EF004012C0E826F5EEC99
:102930000EF0BDEC2BF02FC500F160EC2BF033C195
:1029400082F40401300E82275EEC0EF0A6EF1BF03D
:102950005FEF32F004014C0E826F5EEC0EF004016A
:10296000630E826F5EEC0EF045EC2CF004012C0E31
:10297000826F5EEC0EF0BFEC14F0A6EF1BF0BDEC26
:102980002BF0B5C500F10101003B0F0E001760EC04
:102990002BF033C182F40401300E82275EEC0EF07E
:1029A000B5C500F101010F0E0101001760EC2BF01D
:1029B00033C182F40401300E82275EEC0EF0040174
:1029C0002D0E826F5EEC0EF0B4C500F10101003BEC
:1029D0000F0E001760EC2BF033C182F40401300EAF
:1029E00082275EEC0EF0B4C500F101010F0E01016B
:1029F000001760EC2BF033C182F40401300E822703
:102A00005EEC0EF004012D0E826F5EEC0EF0B3C58D
:102A100000F10101003B0F0E001760EC2BF033C1F9
:102A200082F40401300E82275EEC0EF0B3C500F193
:102A300001010F0E0101001760EC2BF033C182F48D
:102A40000401300E82275EEC0EF00401200E826F2E
:102A50005EEC0EF0B2C500F10F0E0101001760EC44
:102A60002BF033C182F40401300E82275EEC0EF0AD
:102A70000401200E826F5EEC0EF0B1C500F1010181
:102A80000101003B0F0E001760EC2BF033C182F404
:102A90000401300E82275EEC0EF0B1C500F1010199
:102AA0000F0E0101001760EC2BF033C182F404011A
:102AB000300E82275EEC0EF004013A0E826F5EEC5F
:102AC0000EF0B0C500F10101003B0F0E001760ECE5
:102AD0002BF033C182F40401300E82275EEC0EF03D
:102AE000B0C500F101010F0E0101001760EC2BF0E1
:102AF00033C182F40401300E82275EEC0EF0040133
:102B00003A0E826F5EEC0EF0AFC500F10101003BA2
:102B10000F0E001760EC2BF033C182F40401300E6D
:102B200082275EEC0EF0AFC500F101010F0E001719
:102B300060EC2BF033C182F40401300E82275EEC8E
:102B40000EF0120084C3E8FF0F0BE83AE8CFB5F5AA
:102B500085C3E8FF0F0B0501B51387C3E8FF0F0B13
:102B6000E83AE8CFB4F588C3E8FF0F0B0501B413CA
:102B70008AC3E8FF0F0BE83AE8CFB3F58BC3E8FF51
:102B80000F0B0501B3138DC3E8FF0F0BE8CFB2F5B0
:102B90008FC3E8FF0F0BE83AE8CFB1F590C3E8FF29
:102BA0000F0B0501B11392C3E8FF0F0BE83AE8CF12
:102BB000B0F593C3E8FF0F0B0501B01395C3E8FF11
:102BC0000F0BE83AE8CFAFF596C3E8FF0F0B05010E
:102BD000AF13A0EC2CF004014C0E826F5EEC0EF0F3
:102BE0000401430E826F5EEC0EF0B4EF14F0078424
:102BF00004014C0E826F5EEC0EF00401370E826F02
:102C00005EEC0EF004012C0E826F5EEC0EF00501FE
:102C10002E51130A06E005012E51170A0DE092EF1E
:102C200016F00101000E006F000E016F100E026F12
:102C3000000E036F25EF16F00101000E006F000E6D
:102C4000016F000E026F010E036F60EC2BF02AC1C2
:102C500082F40401300E82275EEC0EF02BC182F468
:102C60000401300E82275EEC0EF02CC182F40401C8
:102C7000300E82275EEC0EF02DC182F40401300E7E
:102C800082275EEC0EF02EC182F40401300E822702
:102C90005EEC0EF02FC182F40401300E82275EEC50
:102CA0000EF030C182F40401300E82275EEC0EF08B
:102CB00031C182F40401300E82275EEC0EF032C185
:102CC00082F40401300E82275EEC0EF033C182F4F0
:102CD0000401300E82275EEC0EF004012C0E826F90
:102CE0005EEC0EF00101100E006F000E016F000E81
:102CF000026F000E036F60EC2BF031C182F404010F
:102D0000300E82275EEC0EF032C182F40401300EE8
:102D100082275EEC0EF033C182F40401300E82276C
:102D20005EEC0EF00794A6EF1BF00501216B226B01
:102D3000236B246B04014C0E826F5EEC0EF00401D9
:102D4000380E826F5EEC0EF004012C0E826F5EEC8A
:102D50000EF00101100E006F000E016F000E026FE9
:102D6000000E036F60EC2BF02AC182F40401300ED8
:102D700082275EEC0EF02BC182F40401300E822714
:102D80005EEC0EF02CC182F40401300E82275EEC62
:102D90000EF02DC182F40401300E82275EEC0EF09D
:102DA0002EC182F40401300E82275EEC0EF02FC19A
:102DB00082F40401300E82275EEC0EF030C182F402
:102DC0000401300E82275EEC0EF031C182F4040162
:102DD000300E82275EEC0EF032C182F40401300E18
:102DE00082275EEC0EF033C182F40401300E82279C
:102DF0005EEC0EF004012C0E826F5EEC0EF025C529
:102E000000F126C501F127C502F128C503F1010132
:102E1000100E046F000E056F000E066F000E076F98
:102E2000F3EC2AF000C133F501C134F502C135F5E8
:102E300003C136F560EC2BF02AC182F40401300E98
:102E400082275EEC0EF02BC182F40401300E822743
:102E50005EEC0EF02CC182F40401300E82275EEC91
:102E60000EF02DC182F40401300E82275EEC0EF0CC
:102E70002EC182F40401300E82275EEC0EF02FC1C9
:102E800082F40401300E82275EEC0EF030C182F431
:102E90000401300E82275EEC0EF031C182F4040191
:102EA000300E82275EEC0EF032C182F40401300E47
:102EB00082275EEC0EF033C182F40401300E8227CB
:102EC0005EEC0EF068EC0EF0050133676FEF17F063
:102ED00034676FEF17F035676FEF17F0366702D082
:102EE0000DEF18F0129E21C500F122C501F123C596
:102EF00002F124C503F1899A400EC76E200EC66EFA
:102F00009E96C69E0B0EC96EFF0E9EB602D0E82E90
:102F1000FCD79E96C69E02C1C9FFFF0E9EB602D088
:102F2000E82EFCD79E96C69E01C1C9FFFF0E9EB635
:102F300002D0E82EFCD79E96C69E00C1C9FFFF0EA8
:102F40009EB602D0E82EFCD79E96C69EC952FF0EB2
:102F50009EB602D0E82EFCD70501100E326F040198
:102F600014EE00F080517F0BE1269E96C69EC9525A
:102F7000FF0E9EB602D0E82EFCD7C9CFE7FF0401B2
:102F8000802B0501322FAFEF17F0898A33C500F18E
:102F900034C501F135C502F136C503F10101010E59
:102FA000046F000E056F000E066F000E076FC2EC77
:102FB0002AF000C133F501C134F502C135F503C172
:102FC00036F505013367ECEF17F03467ECEF17F0D7
:102FD0003567ECEF17F0366702D00DEF18F021C51A
:102FE00000F122C501F123C502F124C503F101015D
:102FF000100E046F000E056F000E066F000E076FB7
:10300000C7EC2AF000C121F501C122F502C123F568
:1030100003C124F5128EFDEF24F00401450E826FEA
:103020005EEC0EF004014F0E826F5EEC0EF00401B8
:10303000460E826F5EEC0EF0A6EF1BF0078420ECCC
:1030400032F0BDEC2BF02DC500F160EC2BF004014B
:103050004C0E826F5EEC0EF00401300E826F5EEC5F
:103060000EF004012C0E826F5EEC0EF031C182F482
:103070000401300E82275EEC0EF032C182F40401AE
:10308000300E82275EEC0EF033C182F40401300E64
:1030900082275EEC0EF004012C0E826F5EEC0EF0C7
:1030A000BDEC2BF02EC500F160EC2BF031C182F4A9
:1030B0000401300E82275EEC0EF032C182F404016E
:1030C000300E82275EEC0EF033C182F40401300E24
:1030D00082275EEC0EF00794A6EF1BF004014C0E65
:1030E000826F5EEC0EF00401650E826F5EEC0EF0F6
:1030F00047EC2EF0A6EF1BF004014C0E826F5EEC45
:103100000EF00401450E826F5EEC0EF05EEC2EF0C8
:10311000A6EF1BF004014C0E826F5EEC0EF0040172
:10312000620E826F5EEC0EF08CEC2EF0A6EF1BF0C0
:1031300004014C0E826F5EEC0EF00401420E826FB1
:103140005EEC0EF075EC2EF0A6EF1BF004014C0EB9
:10315000826F5EEC0EF00401760E826F5EEC0EF074
:1031600004012C0E826F5EEC0EF010A807D0040153
:10317000310E826F5EEC0EF0A6EF1BF00401300EF4
:10318000826F5EEC0EF0A6EF1BF004014C0E826F16
:103190005EEC0EF004015A0E826F5EEC0EF004013C
:1031A0002C0E826F5EEC0EF020EC32F0BDEC2BF0BA
:1031B00005012E51130A06E005012E51170A0DE0F4
:1031C000F6EF18F00101000E006F000E016F100EF7
:1031D000026F000E036FF6EF18F00101000E006F92
:1031E000000E016F000E026F010E036F0101100E41
:1031F000046F000E056F000E066F000E076FF3ECF4
:103200002AF060EC2BF02AC182F40401300E8227F0
:103210005EEC0EF02BC182F40401300E82275EECCE
:103220000EF02CC182F40401300E82275EEC0EF009
:103230002DC182F40401300E82275EEC0EF02EC107
:1032400082F40401300E82275EEC0EF02FC182F46E
:103250000401300E82275EEC0EF030C182F40401CE
:10326000300E82275EEC0EF031C182F40401300E84
:1032700082275EEC0EF032C182F40401300E822708
:103280005EEC0EF033C182F40401300E82275EEC56
:103290000EF0A6EF1BF0078404014C0E826F5EEC6B
:1032A0000EF00401310E826F5EEC0EF004012C0E64
:1032B000826F5EEC0EF025C500F126C501F127C531
:1032C00002F128C503F10101100E046F000E056F15
:1032D000000E066F000E076FF3EC2AF060EC2BF087
:1032E0002AC182F40401300E82275EEC0EF02BC15D
:1032F00082F40401300E82275EEC0EF02CC182F4C1
:103300000401300E82275EEC0EF02DC182F4040120
:10331000300E82275EEC0EF02EC182F40401300ED6
:1033200082275EEC0EF02FC182F40401300E82275A
:103330005EEC0EF030C182F40401300E82275EECA8
:103340000EF031C182F40401300E82275EEC0EF0E3
:1033500032C182F40401300E82275EEC0EF033C1DC
:1033600082F40401300E82275EEC0EF00794A6EF83
:103370001BF0078404014C0E826F5EEC0EF004011A
:10338000320E826F5EEC0EF07AEC30F00794A6EF0E
:103390001BF0078404014C0E826F5EEC0EF00401FA
:1033A000330E826F5EEC0EF0D7EC30F0079456EFE0
:1033B00019F0078404014C0E826F5EEC0EF00401DC
:1033C000340E826F5EEC0EF004012C0E826F5EEC08
:1033D0000EF0FEEC2BF084C32AF185C32BF186C3DB
:1033E0002CF187C32DF188C32EF189C32FF18AC335
:1033F00030F18BC331F18CC332F18DC333F1010154
:10340000296B0BEC2CF082EC2BF0100E046F000EED
:10341000056F000E066F000E076FD3EC2AF000C197
:1034200021F501C122F502C123F503C124F5D3EC36
:1034300031F038C5AFF539C5B0F53AC5B1F53BC582
:10344000B2F53CC5B3F53DC5B4F53EC5B5F5BFEC29
:1034500014F004012C0E826F5EEC0EF03FC500F1FB
:1034600040C501F141C502F142C503F10101000E61
:10347000046F000E056F010E066F000E076FF3EC70
:103480002AF060EC2BF0296748EF1AF04DEF1AF0A4
:1034900004012D0E826F5EEC0EF030C182F4040147
:1034A000300E82275EEC0EF031C182F40401300E42
:1034B00082275EEC0EF004012E0E826F5EEC0EF0A1
:1034C00032C182F40401300E82275EEC0EF033C16B
:1034D00082F40401300E82275EEC0EF004012C0E03
:1034E000826F5EEC0EF0BDEC2BF043C500F144C5DD
:1034F00001F127EC26F004012C0E826F5EEC0EF039
:10350000BDEC2BF045C500F160EC2BF031C182F42D
:103510000401300E82275EEC0EF032C182F4040109
:10352000300E82275EEC0EF033C182F40401300EBF
:1035300082275EEC0EF00794A6EF1BF0FEEC2BF05A
:1035400085C32AF186C32BF187C32CF188C32DF1E3
:1035500089C32EF18AC32FF18BC330F18CC331F1B3
:103560008DC332F18EC333F10101296B0BEC2CF0CA
:1035700082EC2BF00101010E046F000E056F000EAE
:10358000066F000E076FC2EC2AF0100E046F000EDB
:10359000056F000E066F000E076FD3EC2AF000C116
:1035A00029F501C12AF502C12BF503C12CF501EC67
:1035B00030F004014C0E826F5EEC0EF00401460EFA
:1035C000826F5EEC0EF004012C0E826F5EEC0EF04A
:1035D00025C500F126C501F127C502F128C503F173
:1035E0000101100E046F000E056F000E066F000E35
:1035F000076FF3EC2AF060EC2BF02AC182F404018F
:10360000300E82275EEC0EF02BC182F40401300EE6
:1036100082275EEC0EF02CC182F40401300E82276A
:103620005EEC0EF02DC182F40401300E82275EECB8
:103630000EF02EC182F40401300E82275EEC0EF0F3
:103640002FC182F40401300E82275EEC0EF030C1EF
:1036500082F40401300E82275EEC0EF031C182F458
:103660000401300E82275EEC0EF032C182F40401B8
:10367000300E82275EEC0EF033C182F40401300E6E
:1036800082275EEC0EF0A6EF1BF00F98D7EC30F01F
:10369000FDEF24F004014C0E826F5EEC0EF004018D
:1036A000350E826F5EEC0EF004012C0E826F5EEC24
:1036B0000EF0BDEC2BF00784B9C500F1079460EC67
:1036C0002BF031C182F40401300E82275EEC0EF043
:1036D00032C182F40401300E82275EEC0EF033C159
:1036E00082F40401300E82275EEC0EF0A6EF1BF090
:1036F0009AEC30F0BDEC2BF037C500F160EC2BF00C
:1037000004014C0E826F5EEC0EF00401360E826FE7
:103710005EEC0EF004012C0E826F5EEC0EF031C1F7
:1037200082F40401300E82275EEC0EF032C182F486
:103730000401300E82275EEC0EF033C182F40401E6
:10374000300E82275EEC0EF0A6EF1BF068EC0EF058
:10375000FDEF24F004014C0E826F5EEC0EF00401CC
:10376000500E826F5EEC0EF004012C0E826F5EEC48
:103770000EF085C32AF186C32BF187C32CF188C3D1
:103780002DF189C32EF18AC32FF18BC330F18CC385
:1037900031F18DC332F18EC333F101010BEC2CF00A
:1037A00082EC2BF003018451530A0DE00301845194
:1037B0004D0A38E00401780E826F5EEC0EF068EC82
:1037C0000EF0FDEF24F00401530E826F5EEC0EF05C
:1037D000250E0C6E00C10BF002EC0BF0260E0C6EE9
:1037E00001C10BF002EC0BF0270E0C6E02C10BF0C6
:1037F00002EC0BF0280E0C6E03C10BF002EC0BF088
:1038000000C157F501C158F502C159F503C15AF578
:1038100000C15BF501C15CF502C15DF503C15EF558
:1038200087EF1CF004014D0E826F5EEC0EF0290E46
:103830000C6E00C10BF002EC0BF000C15FF500C193
:1038400060F587EF1CF004014C0E826F5EEC0EF009
:103850000401540E826F5EEC0EF004012C0E826F98
:103860005EEC0EF084C32AF185C32BF186C32CF1E4
:1038700087C32DF188C32EF189C32FF18AC330F19C
:103880008BC331F18DC332F18EC333F101010BECE7
:103890002CF082EC2BF00101000E046F000E056F7E
:1038A000010E066F000E076FD3EC2AF0210E0C6E8E
:1038B00000C10BF002EC0BF0220E0C6E01C10BF0FC
:1038C00002EC0BF0230E0C6E02C10BF002EC0BF0BD
:1038D000240E0C6E03C10BF002EC0BF000C161F57D
:1038E00001C162F502C163F503C164F587EF1CF005
:1038F00004014C0E826F5EEC0EF00401490E826FE3
:103900005EEC0EF004012C0E826F5EEC0EF0250EC4
:1039100019EC0BF0E8CF00F1260E19EC0BF0E8CF14
:1039200001F1270E19EC0BF0E8CF02F1280E19EC8B
:103930000BF0E8CF03F160EC2BF043EC29F004012D
:10394000730E826F5EEC0EF004012C0E826F5EEC43
:103950000EF0BDEC2BF0290E19EC0BF0E8CF00F1C6
:1039600060EC2BF043EC29F00401730E826F5EECE7
:103970000EF004012C0E826F5EEC0EF05BC500F1C0
:103980005CC501F15DC502F15EC503F160EC2BF091
:1039900043EC29F00401730E826F5EEC0EF004011B
:1039A0002C0E826F5EEC0EF0BDEC2BF060C500F1CA
:1039B00060EC2BF043EC29F004016D0E826F5EEC9D
:1039C0000EF004012C0E826F5EEC0EF061C500F16A
:1039D00062C501F163C502F164C503F118EC25F07D
:1039E00004012C0E826F5EEC0EF068EC0EF0FDEF21
:1039F00024F083C32AF184C32BF185C32CF186C341
:103A00002DF187C32EF188C32FF189C330F18AC30A
:103A100031F18BC332F18CC333F101010BEC2CF08B
:103A200082EC2BF0160E0C6E00C10BF002EC0BF0CA
:103A3000170E0C6E01C10BF002EC0BF0180E0C6EA1
:103A400002C10BF002EC0BF0190E0C6E03C10BF06F
:103A500002EC0BF000C18AF101C18BF102C18CF1C3
:103A600003C18DF100C18EF101C18FF102C190F14E
:103A700003C191F1DBEF1DF083C32AF184C32BF165
:103A800085C32CF186C32DF187C32EF188C32FF196
:103A900089C330F18AC331F18BC332F18CC333F166
:103AA00001010BEC2CF082EC2BF000C18AF101C17A
:103AB0008BF102C18CF103C18DF100C18EF101C106
:103AC0008FF102C190F103C191F1DBEF1DF083C3CF
:103AD0002AF184C32BF185C32CF186C32DF187C352
:103AE0002EF188C32FF189C330F18AC331F18CC321
:103AF00032F18DC333F101010BEC2CF082EC2BF091
:103B00000101000E046F000E056F010E066F000E1E
:103B1000076FD3EC2AF01A0E0C6E00C10BF002EC0A
:103B20000BF01B0E0C6E01C10BF002EC0BF01C0E27
:103B30000C6E02C10BF002EC0BF01D0E0C6E03C1FB
:103B40000BF002EC0BF000C192F101C193F102C144
:103B500094F103C195F1DBEF1DF083C32AF184C317
:103B60002BF185C32CF186C32DF187C32EF188C3B9
:103B70002FF189C330F18AC331F18CC332F18DC387
:103B800033F101010BEC2CF082EC2BF00101000E63
:103B9000046F000E056F010E066F000E076FD3EC69
:103BA0002AF000C192F101C193F102C194F103C165
:103BB00095F1DBEF1DF0160E19EC0BF0E8CF00F1DC
:103BC000170E19EC0BF0E8CF01F1180E19EC0BF001
:103BD000E8CF02F1190E19EC0BF0E8CF03F160EC1D
:103BE0002BF043EC29F00401730E826F5EEC0EF0B3
:103BF00004012C0E826F5EEC0EF08AC100F18BC1C5
:103C000001F18CC102F18DC103F160EC2BF043ECAA
:103C100029F00401730E826F5EEC0EF004012C0E8D
:103C2000826F5EEC0EF01A0E19EC0BF0E8CF00F18B
:103C30001B0E19EC0BF0E8CF01F11C0E19EC0BF088
:103C4000E8CF02F11D0E19EC0BF0E8CF03F118ECF0
:103C500025F004012C0E826F5EEC0EF092C100F193
:103C600093C101F194C102F195C103F118EC25F063
:103C700068EC0EF0FDEF24F00401690E826F5EEC3B
:103C80000EF004012C0E826F5EEC0EF00101040EAA
:103C9000006F000E016F000E026F000E036F60ECEC
:103CA0002BF02CC182F40401300E82275EEC0EF062
:103CB0002DC182F40401300E82275EEC0EF02EC17D
:103CC00082F40401300E82275EEC0EF02FC182F4E4
:103CD0000401300E82275EEC0EF030C182F4040144
:103CE000300E82275EEC0EF031C182F40401300EFA
:103CF00082275EEC0EF032C182F40401300E82277E
:103D00005EEC0EF033C182F40401300E82275EECCB
:103D10000EF004012C0E826F5EEC0EF00101060E17
:103D2000006F000E016F000E026F000E036F60EC5B
:103D30002BF02CC182F40401300E82275EEC0EF0D1
:103D40002DC182F40401300E82275EEC0EF02EC1EC
:103D500082F40401300E82275EEC0EF02FC182F453
:103D60000401300E82275EEC0EF030C182F40401B3
:103D7000300E82275EEC0EF031C182F40401300E69
:103D800082275EEC0EF032C182F40401300E8227ED
:103D90005EEC0EF033C182F40401300E82275EEC3B
:103DA0000EF004012C0E826F5EEC0EF001012D0E60
:103DB000006F000E016F000E026F000E036F60ECCB
:103DC0002BF02CC182F40401300E82275EEC0EF041
:103DD0002DC182F40401300E82275EEC0EF02EC15C
:103DE00082F40401300E82275EEC0EF02FC182F4C3
:103DF0000401300E82275EEC0EF030C182F4040123
:103E0000300E82275EEC0EF031C182F40401300ED8
:103E100082275EEC0EF032C182F40401300E82275C
:103E20005EEC0EF033C182F40401300E82275EECAA
:103E30000EF004012C0E826F5EEC0EF0200EF86E78
:103E4000F76AF66A04010900F5CF82F45EEC0EF021
:103E50000900F5CF82F45EEC0EF00900F5CF82F494
:103E60005EEC0EF00900F5CF82F45EEC0EF0090076
:103E7000F5CF82F45EEC0EF00900F5CF82F45EEC33
:103E80000EF00900F5CF82F45EEC0EF00900F5CFDC
:103E900082F45EEC0EF068EC0EF0FDEF24F083513E
:103EA000630AD8A4FDEF24F08451610AD8A4FDEF81
:103EB00024F085516C0AD8A4FDEF24F08651410A04
:103EC0003FE08651440A1BE08651420AD8B4B3EF62
:103ED0001FF08651350AD8B487EF26F08651360A8E
:103EE000D8B4DCEF26F08651370AD8B445EF27F076
:103EF0008651380AD8B4A3EF27F0FDEF24F00798D5
:103F0000079A04017A0E826F5EEC0EF00401780EBF
:103F1000826F5EEC0EF00401640E826F5EEC0EF0B8
:103F20000401550E826F5EEC0EF09CEF1FF0040151
:103F30004C0E826F5EEC0EF068EC0EF0FDEF24F09C
:103F40000788079A04017A0E826F5EEC0EF0040176
:103F5000410E826F5EEC0EF00401610E826F5EEC2A
:103F60000EF090EF1FF00798078A04017A0E826F17
:103F70005EEC0EF00401420E826F5EEC0EF0040166
:103F8000610E826F5EEC0EF090EF1FF0010166672C
:103F9000D1EF1FF06767D1EF1FF06867D1EF1FF017
:103FA000696715D04F67DCEF1FF05067DCEF1FF03B
:103FB0005167DCEF1FF052670AD00101000E006F5D
:103FC000000E016F000E026F000E036F120011B899
:103FD0000AD00101620E046F010E056F000E066F1C
:103FE000000E076F09D00101A70E046F020E056FC6
:103FF000000E066F000E076F66C100F167C101F188
:1040000068C102F169C103F1C2EC2AF003BF79EF84
:1040100020F0119A119C0101000E046FA80E056F8B
:10402000550E066F020E076F66C100F167C101F100
:1040300068C102F169C103F166C186F167C187F108
:1040400068C188F169C189F1C2EC2AF003BF0BD0C5
:104050000101000E866FA80E876F550E886F020E45
:10406000896F118A119C0E0E19EC0BF0E8CF18F134
:104070000F0E19EC0BF0E8CF19F1100E19EC0BF044
:10408000E8CF1AF1110E19EC0BF0E8CF1BF10BEC95
:104090002AF086C104F187C105F188C106F189C102
:1040A00007F1C2EC2AF00782CFEC29F00BEC2AF0E2
:1040B0000792CFEC29F086C100F187C101F188C1D8
:1040C00002F189C103F10792CFEC29F0CC0E046F05
:1040D000E00E056F870E066F050E076FC2EC2AF023
:1040E00000C118F101C119F102C11AF103C11BF19C
:1040F0003BD0119C119A0101800E006F1A0E016FC6
:10410000060E026F000E036F4FC104F150C105F19E
:1041100051C106F152C107F1C2EC2AF003AF05D03C
:10412000BDEC2BF0118C119A12000E0E19EC0BF055
:10413000E8CF18F10F0E19EC0BF0E8CF19F1100EC3
:1041400019EC0BF0E8CF1AF1110E19EC0BF0E8CFD7
:104150001BF14FC100F150C101F151C102F152C137
:1041600003F10782CFEC29F018C100F119C101F168
:104170001AC102F11BC103F112000401730E826F18
:104180005EEC0EF004012C0E826F5EEC0EF00784E4
:1041900062C166F163C167F164C168F165C169F12B
:1041A0004BC14FF14CC150F14DC151F14EC152F1D3
:1041B00057C159F158C15AF10794E3EC20F068EC6B
:1041C0000EF0FDEF24F066C100F167C101F168C196
:1041D00002F169C103F1010160EC2BF043EC29F01D
:1041E0000401630E826F5EEC0EF004012C0E826FF0
:1041F0005EEC0EF04FC100F150C101F151C102F16E
:1042000052C103F1010160EC2BF043EC29F00401F1
:10421000660E826F5EEC0EF004012C0E826F5EEC77
:104220000EF0BDEC2BF059C100F15AC101F10101B2
:1042300060EC2BF043EC29F00401740E826F5EEC0D
:104240000EF0120010820401530E826F5EEC0EF02D
:1042500004012C0E826F5EEC0EF083C32AF184C33E
:104260002BF185C32CF186C32DF187C32EF188C3B2
:104270002FF189C330F18AC331F18BC332F18CC382
:1042800033F101010BEC2CF082EC2BF000C166F154
:1042900001C167F102C168F103C169F18EC32AF15E
:1042A0008FC32BF190C32CF191C32DF192C32EF14A
:1042B00093C32FF194C330F195C331F196C332F11A
:1042C00097C333F101010BEC2CF082EC2BF000C111
:1042D0004FF101C150F102C151F103C152F1FEECA5
:1042E0002BF099C32FF19AC330F19BC331F19CC3DA
:1042F00032F19DC333F101010BEC2CF082EC2BF079
:1043000000C159F101C15AF1E3EC20F004012C0E77
:10431000826F5EEC0EF09CEF21F0118E18A002D09F
:1043200018AE108C17BE02D017A4108E8251520AFC
:1043300002E10F8201D00F928251750A02E11084CE
:1043400001D010948251550A02E1108601D01096D6
:1043500011A003D011A401D01084078410B20AEF79
:1043600022F010A4F6EF21F0B6C166F1B7C167F1F3
:10437000B8C168F1B9C169F1BAC16AF1BBC16BF1E9
:10438000BCC16CF1BDC16DF1BEC16EF1BFC16FF1B9
:10439000C0C170F1C1C171F1C2C172F1C3C173F189
:1043A000C4C174F1C5C175F1C6C176F1C7C177F159
:1043B000C8C178F1C9C179F1CAC17AF1CBC17BF129
:1043C000CCC17CF1CDC17DF1CEC17EF1CFC17FF1F9
:1043D000D0C180F1D1C181F1D2C182F1D3C183F1C9
:1043E000D4C184F1D5C185F1FEEF21F062C166F13F
:1043F00063C167F164C168F165C169F14BC14FF1F7
:104400004CC150F14DC151F14EC152F157C159F15A
:1044100058C15AF107940FA02CEF22F001019267C6
:1044200019EF22F0936719EF22F0946719EF22F049
:1044300095671DEF22F02CEF22F0C6EC1FF092C121
:1044400004F193C105F194C106F195C107F1C2ECE5
:104450002AF003BFC3EF24F0C6EC1FF00101000EE9
:10446000046F000E056F010E066F000E076FF3EC70
:104470002AF011A02CD011A22AD060EC2BF02967D1
:1044800001D007D004012D0E826F5EEC0EF0C1EF5B
:1044900024F030C182F40401300E82275EEC0EF06D
:1044A00031C182F40401300E82275EEC0EF032C17D
:1044B00082F40401300E82275EEC0EF033C182F4E8
:1044C0000401300E82275EEC0EF0C1EF24F012A83A
:1044D000C5D0129819C01AF01A3A1A42070E1A16C5
:1044E00000011A50000AD8B4FAEF22F000011A5065
:1044F000010AD8B486EF22F000011A50020AD8B49B
:1045000084EF22F02CEF23F02CEF23F0BDEC2BF006
:1045100029C001F12AC000F1D89001330033D890AE
:10452000013300330101630E046F000E056F000EAE
:10453000066F000E076FF3EC2AF0280E046F000ED2
:10454000056F000E066F000E076FC2EC2AF000C167
:104550002CF0BDEC2BF027C001F1019F019D28C07C
:1045600000F10101A40E046F000E056F000E066F2E
:10457000000E076FF3EC2AF000C12BF000C104F12C
:1045800001C105F102C106F103C107F1640E006F1C
:10459000000E016F000E026F000E036FC2EC2AF0D6
:1045A000050E046F000E056F000E066F000E076FFC
:1045B000F3EC2AF000C104F101C105F102C106F1DA
:1045C00003C107F1BDEC2BF02CC000F1C2EC2AF0C6
:1045D00000C12DF02DC0E8FF050F2C5C03E78A8495
:1045E0002CEF23F02DC0E8FF0A0F2C5C01E68A9423
:1045F0002CEF23F000C124F101C125F102C126F105
:1046000003C127F1BDEC2BF0C3EC2BF019501F0BAD
:10461000E8CF00F10101640E046F000E056F000E7B
:10462000066F000E076FD3EC2AF024C104F125C1F8
:1046300005F126C106F127C107F1C2EC2AF003BF3C
:1046400002D08A9401D08A8424C100F125C101F1ED
:1046500026C102F127C103F1C3EF24F000C124F108
:1046600001C125F102C126F103C127F110AE4CD0E2
:10467000109E00C108F101C109F102C10AF103C194
:104680000BF160EC2BF030C1D6F131C1D7F132C162
:10469000D8F133C1D9F108C100F109C101F10AC152
:1046A00002F10BC103F101016C0E046F070E056FDF
:1046B000000E066F000E076FC2EC2AF003BF04D095
:1046C0000101550EDA6F1CD008C100F109C101F1DA
:1046D0000AC102F10BC103F10101A40E046F060E21
:1046E000056F000E066F000E076FC2EC2AF003BFC5
:1046F00004D001017F0EDA6F03D00101FF0EDA6FE3
:104700001B8E11AEC3EF24F024C100F125C101F1CD
:1047100026C102F127C103F110A496EF23F0040192
:10472000750E826F5EEC0EF09BEF23F00401720EAB
:10473000826F5EEC0EF004012C0E826F5EEC0EF0C8
:1047400060EC2BF02967AAEF23F00401200E826FA2
:10475000ADEF23F004012D0E826F5EEC0EF030C140
:1047600082F40401300E82275EEC0EF031C182F437
:104770000401300E82275EEC0EF004012E0E826FD3
:104780005EEC0EF032C182F40401300E82275EEC42
:104790000EF033C182F40401300E82275EEC0EF07D
:1047A00004016D0E826F5EEC0EF004012C0E826F20
:1047B0005EEC0EF04FC100F150C101F151C102F1A8
:1047C00052C103F1010160EC2BF043EC29F004012C
:1047D000480E826F5EEC0EF004017A0E826F5EEC82
:1047E0000EF004012C0E826F5EEC0EF066C100F13B
:1047F00067C101F168C102F169C103F1010160EC17
:104800002BF043EC29F00401630E826F5EEC0EF096
:1048100004012C0E826F5EEC0EF066C100F167C1E0
:1048200001F168C102F169C103F101010A0E046FCF
:10483000000E056F000E066F000E076FD3EC2AF016
:10484000000E046F120E056F000E066F000E076F4C
:10485000F3EC2AF060EC2BF02AC182F40401300E54
:1048600082275EEC0EF02BC182F40401300E822709
:104870005EEC0EF02CC182F40401300E82275EEC57
:104880000EF02DC182F40401300E82275EEC0EF092
:104890002EC182F40401300E82275EEC0EF02FC18F
:1048A00082F40401300E82275EEC0EF030C182F4F7
:1048B0000401300E82275EEC0EF004012E0E826F92
:1048C0005EEC0EF031C182F40401300E82275EEC02
:1048D0000EF032C182F40401300E82275EEC0EF03D
:1048E00033C182F40401300E82275EEC0EF0040125
:1048F000730E826F5EEC0EF004012C0E826F5EEC84
:104900000EF0BDEC2BF059C100F15AC101F127ECBA
:1049100026F00FB28FEF24F00FA0C1EF24F00401B6
:104920002C0E826F5EEC0EF0200EF86EF76AF66ABF
:1049300004010900F5CF82F45EEC0EF00900F5CF1A
:1049400082F45EEC0EF00900F5CF82F45EEC0EF01E
:104950000900F5CF82F45EEC0EF00900F5CF82F489
:104960005EEC0EF00900F5CF82F45EEC0EF009006B
:10497000F5CF82F45EEC0EF00900F5CF82F45EEC28
:104980000EF068EC0EF00F90FDEF24F00401630EC2
:10499000826F5EEC0EF004012C0E826F5EEC0EF066
:1049A00003EC25F004012C0E826F5EEC0EF076EC29
:1049B00025F004012C0E826F5EEC0EF0F2EC25F077
:1049C00004012C0E826F5EEC0EF00101F80E006FF8
:1049D000CD0E016F660E026F030E036F18EC25F00B
:1049E00004012C0E826F5EEC0EF008EC26F068ECF1
:1049F0000EF0FDEF24F068EC0EF00301C26B07909F
:104A000010920CEF28F0D8900E0E19EC0BF0E8CFB6
:104A100000F10F0E19EC0BF0E8CF01F1100E19ECBC
:104A20000BF0E8CF02F1110E19EC0BF0E8CF03F117
:104A30000101000E046F000E056F010E066F000EDF
:104A4000076FF3EC2AF060EC2BF02AC182F404012A
:104A5000300E82275EEC0EF02BC182F40401300E82
:104A600082275EEC0EF02CC182F40401300E822706
:104A70005EEC0EF02DC182F40401300E82275EEC54
:104A80000EF02EC182F40401300E82275EEC0EF08F
:104A90002FC182F40401300E82275EEC0EF030C18B
:104AA00082F40401300E82275EEC0EF031C182F4F4
:104AB0000401300E82275EEC0EF004012E0E826F90
:104AC0005EEC0EF032C182F40401300E82275EECFF
:104AD0000EF033C182F40401300E82275EEC0EF03A
:104AE00004016D0E826F5EEC0EF01200120E19ECD6
:104AF0000BF0E8CF00F1130E19EC0BF0E8CF01F149
:104B0000140E19EC0BF0E8CF02F1150E19EC0BF0B6
:104B1000E8CF03F101010A0E046F000E056F000ECD
:104B2000066F000E076FD3EC2AF0000E046F120E12
:104B3000056F000E066F000E076FF3EC2AF060ECB5
:104B40002BF02AC182F40401300E82275EEC0EF0B5
:104B50002BC182F40401300E82275EEC0EF02CC1D2
:104B600082F40401300E82275EEC0EF02DC182F437
:104B70000401300E82275EEC0EF02EC182F4040197
:104B8000300E82275EEC0EF02FC182F40401300E4D
:104B900082275EEC0EF030C182F40401300E8227D1
:104BA0005EEC0EF004012E0E826F5EEC0EF031C151
:104BB00082F40401300E82275EEC0EF032C182F4E2
:104BC0000401300E82275EEC0EF033C182F4040142
:104BD000300E82275EEC0EF00401730E826F5EECE5
:104BE0000EF012000A0E19EC0BF0E8CF00F10B0EDC
:104BF00019EC0BF0E8CF01F10C0E19EC0BF0E8CF3B
:104C000002F10D0E19EC0BF0E8CF03F127EF26F0BF
:104C1000060E19EC0BF0E8CF00F1070E19EC0BF0C3
:104C2000E8CF01F1080E19EC0BF0E8CF02F1090E04
:104C300019EC0BF0E8CF03F127EF26F00101BDECF2
:104C40002BF0078457C100F158C101F1079401010D
:104C5000E80E046F800E056F000E066F000E076FE2
:104C6000D3EC2AF0000E046F040E056F000E066FE1
:104C7000000E076FF3EC2AF0880E046F130E056F19
:104C8000000E066F000E076FC2EC2AF00A0E046FCA
:104C9000000E056F000E066F000E076FF3EC2AF092
:104CA00060EC2BF0010129675BEF26F00401200E78
:104CB000826F5EEF26F004012D0E826F5EEC0EF027
:104CC00030C182F40401300E82275EEC0EF031C157
:104CD00082F40401300E82275EEC0EF032C182F4C1
:104CE0000401300E82275EEC0EF004012E0E826F5E
:104CF0005EEC0EF033C182F40401300E82275EECCC
:104D00000EF00401430E826F5EEC0EF0120087C3BA
:104D10002AF188C32BF189C32CF18AC32DF18BC3EF
:104D20002EF18CC32FF18DC330F18EC331F190C3BE
:104D300032F191C333F10101296B0BEC2CF082ECC1
:104D40002BF00101000E046F000E056F010E066FBF
:104D5000000E076FD3EC2AF00E0E0C6E00C10BF0A4
:104D600002EC0BF00F0E0C6E01C10BF002EC0BF01D
:104D7000100E0C6E02C10BF002EC0BF0110E0C6E5B
:104D800003C10BF002EC0BF004017A0E826F5EECB3
:104D90000EF004012C0E826F5EEC0EF00401350E55
:104DA000826F5EEC0EF004012C0E826F5EEC0EF052
:104DB00003EC25F09CEF1FF087C32AF188C32BF189
:104DC00089C32CF18AC32DF18BC32EF18CC32FF133
:104DD0008DC330F18EC331F190C332F191C333F101
:104DE0000101296B0BEC2CF082EC2BF0880E046F88
:104DF000130E056F000E066F000E076FC7EC2AF04A
:104E0000000E046F040E056F000E066F000E076F94
:104E1000D3EC2AF00101E80E046F800E056F000E3E
:104E2000066F000E076FF3EC2AF00A0E0C6E00C13D
:104E30000BF002EC0BF00B0E0C6E01C10BF002EC50
:104E40000BF00C0E0C6E02C10BF002EC0BF00D0E11
:104E50000C6E03C10BF002EC0BF004017A0E826FB2
:104E60005EEC0EF004012C0E826F5EEC0EF004017D
:104E7000360E826F5EEC0EF004012C0E826F5EEC3B
:104E80000EF0F2EC25F09CEF1FF087C32AF188C3E7
:104E90002BF189C32CF18AC32DF18BC32EF18CC366
:104EA0002FF18DC330F18FC331F190C332F191C333
:104EB00033F101010BEC2CF082EC2BF0000E046FAF
:104EC000120E056F000E066F000E076FD3EC2AF06E
:104ED00001010A0E046F000E056F000E066F000E32
:104EE000076FF3EC2AF0120E0C6E00C10BF002EC0F
:104EF0000BF0130E0C6E01C10BF002EC0BF0140E54
:104F00000C6E02C10BF002EC0BF0150E0C6E03C11F
:104F10000BF002EC0BF004017A0E826F5EEC0EF0E7
:104F200004012C0E826F5EEC0EF00401370E826FCE
:104F30005EEC0EF004012C0E826F5EEC0EF076EC4F
:104F400025F09CEF1FF087C32AF188C32BF189C39A
:104F50002CF18AC32DF18BC32EF18CC32FF18DC39D
:104F600030F18EC331F190C332F191C333F10101BD
:104F7000296B0BEC2CF082EC2BF0880E046F130ED7
:104F8000056F000E066F000E076FC7EC2AF0000ECB
:104F9000046F040E056F000E066F000E076FD3EC52
:104FA0002AF00101E80E046F800E056F000E066FF7
:104FB000000E076FF3EC2AF0060E0C6E00C10BF02A
:104FC00002EC0BF0070E0C6E01C10BF002EC0BF0C3
:104FD000080E0C6E02C10BF002EC0BF0090E0C6E09
:104FE00003C10BF002EC0BF004017A0E826F5EEC51
:104FF0000EF004012C0E826F5EEC0EF00401380EF0
:10500000826F5EEC0EF004012C0E826F5EEC0EF0EF
:1050100008EC26F09CEF1FF007A880EF28F00101B4
:10502000800E006F1A0E016F060E026F000E036FE6
:105030004BC104F14CC105F14DC106F14EC107F160
:10504000C2EC2AF003BFC7EF28F03DEC29F04BC1BA
:1050500000F14CC101F14DC102F14EC103F10782D3
:10506000CFEC29F018C104F119C105F11AC106F1FC
:105070001BC107F1F80E006FCD0E016F660E026FB7
:10508000030E036FC2EC2AF00E0E0C6E00C10BF083
:1050900002EC0BF00F0E0C6E01C10BF002EC0BF0EA
:1050A000100E0C6E02C10BF002EC0BF0110E0C6E28
:1050B00003C10BF002EC0BF007840101BDEC2BF0F7
:1050C00057C100F158C101F107940A0E0C6E00C1DE
:1050D0000BF002EC0BF00B0E0C6E01C10BF002ECAE
:1050E0000BF00C0E0C6E02C10BF002EC0BF00D0E6F
:1050F0000C6E03C10BF002EC0BF00798C7EF28F021
:1051000007AAC7EF28F007840101BDEC2BF057C1B7
:1051100000F158C101F10794060E0C6E00C10BF0AE
:1051200002EC0BF0070E0C6E01C10BF002EC0BF061
:10513000080E0C6E02C10BF002EC0BF0090E0C6EA7
:1051400003C10BF002EC0BF0078462C100F163C1F4
:1051500001F164C102F165C103F10794120E0C6EF6
:1051600000C10BF002EC0BF0130E0C6E01C10BF042
:1051700002EC0BF0140E0C6E02C10BF002EC0BF003
:10518000150E0C6E03C10BF002EC0BF0079A040134
:10519000805181197F0B0DE09EA8FED714EE00F020
:1051A00081517F0BE126E750812B0F01AD6EC7EFD8
:1051B00028F005012F51010A13E081AAF0EF28F031
:1051C00005012F51000A0AE00FB8F0EF28F00501A1
:1051D0003067F0EF28F00FB8F0EF28F05FEF32F013
:1051E00081B805EF29F0EDEC2CF005012F51020AF2
:1051F00002E005EF29F0602F05EF29F05FC560F5AB
:105200000501010E306F3C0E316FAFEF0DF018C18C
:1052100000F119C101F11AC102F11BC103F1000E25
:10522000046F000E056F010E066F000E076FF3ECA2
:105230002AF029A132EF29F02051D8B432EF29F019
:1052400018C100F119C101F11AC102F11BC103F12A
:10525000000E046F000E056F0A0E066F000E076F3A
:10526000F3EC2AF01200010104510013055101135F
:10527000065102130751031312000101186B196B39
:105280001A6B1B6B12002AC182F40401300E8227B4
:105290005EEC0EF02BC182F40401300E82275EEC2E
:1052A0000EF02CC182F40401300E82275EEC0EF069
:1052B0002DC182F40401300E82275EEC0EF02EC167
:1052C00082F40401300E82275EEC0EF02FC182F4CE
:1052D0000401300E82275EEC0EF030C182F404012E
:1052E000300E82275EEC0EF031C182F40401300EE4
:1052F00082275EEC0EF032C182F40401300E822768
:105300005EEC0EF033C182F40401300E82275EECB5
:105310000EF012002FC182F40401300E82275EECE1
:105320000EF030C182F40401300E82275EEC0EF0E4
:1053300031C182F40401300E82275EEC0EF032C1DE
:1053400082F40401300E82275EEC0EF033C182F449
:105350000401300E82275EEC0EF01200060E1D6E68
:10536000060E1E6E060E1F6E1D2EB4EF29F01E2EA9
:10537000B4EF29F01F2EB4EF29F08B84020E1D6EBE
:10538000020E1E6E020E1F6E1D2EC4EF29F01E2E81
:10539000C4EF29F01F2EC4EF29F08B9412000101F5
:1053A000005305E1015303E1025301E1002B92ECAC
:1053B0002AF0BDEC2BF03951006F3A51016F420ECB
:1053C000046F4B0E056F000E066F000E076FD3ECD7
:1053D0002AF000C104F101C105F102C106F103C1C7
:1053E00007F118C100F119C101F11AC102F11BC185
:1053F00003F107B200EF2AF0C7EC2AF002EF2AF01F
:10540000C2EC2AF000C118F101C119F102C11AF170
:1054100003C11BF11200BDEC2BF059C100F15AC1C0
:1054200001F1060E19EC0BF0E8CF04F1070E19ECB0
:105430000BF0E8CF05F1080E19EC0BF0E8CF06F100
:10544000090E19EC0BF0E8CF07F1C2EC2AF000C10D
:1054500024F101C125F102C126F103C127F1290E72
:10546000046F000E056F000E066F000E076FD3EC81
:105470002AF0EE0E046F430E056F000E066F000E4D
:10548000076FC7EC2AF024C104F125C105F126C13C
:1054900006F127C107F1D3EC2AF000C11CF101C1CC
:1054A0001DF102C11EF103C11FF1120E19EC0BF028
:1054B000E8CF04F1130E19EC0BF0E8CF05F1140E50
:1054C00019EC0BF0E8CF06F1150E19EC0BF0E8CF54
:1054D00007F10D0E006F000E016F000E026F000E3F
:1054E000036FD3EC2AF0180E046F000E056F000E48
:1054F000066F000E076FF3EC2AF01CC104F11DC10A
:1055000005F11EC106F11FC107F1C7EC2AF06A0EB2
:10551000046F2A0E056F000E066F000E076FC2ECB7
:105520002AF01200BF0EFA6E200E3A6F396BD89037
:105530000037013702370337D8B0A3EF2AF03A2FEC
:1055400098EF2AF039073A070353D8B41200033111
:10555000070B80093F6F03390F0B010F396F80EC88
:105560005FF0406F390580EC5FF0405D405F396B64
:105570003F33D8B0392739333FA9B8EF2AF040512B
:10558000392712000101E2EC2BF0D8B01200010122
:1055900003510719346FA5EC2BF0D890075103196C
:1055A00034AF800F12000101346BC9EC2BF0D8A08E
:1055B000DFEC2BF0D8B01200B4EC2BF0BDEC2BF0EC
:1055C0001F0E366FF5EC2BF00B35D8B0A5EC2BF099
:1055D000D8A00335D8B01200362FE2EF2AF034B14C
:1055E000CCEC2BF012000101346B045105110611B3
:1055F00007110008D8A0C9EC2BF0D8A0DFEC2BF0E5
:10560000D8B01200086B096B0A6B0B6BF5EC2BF032
:105610001F0E366FF5EC2BF007510B5DD8A41DEF74
:105620002BF006510A5DD8A41DEF2BF00551095D42
:10563000D8A41DEF2BF00451085DD8A030EF2BF05B
:105640000451085F0551D8A0053D095F0651D8A057
:10565000063D0A5F0751D8A0073D0B5FD890008137
:10566000362F0AEF2BF034B1CCEC2BF0346BC9ECB5
:105670002BF0D890F9EC2BF007510B5DD8A44DEF2F
:105680002BF006510A5DD8A44DEF2BF00551095DB2
:10569000D8A44DEF2BF00451085DD8A05CEF2BF09F
:1056A000003F5CEF2BF0013F5CEF2BF0023F5CEF23
:1056B0002BF0032BD8B4120034B1CCEC2BF0120039
:1056C0000101346BC9EC2BF0D8B01200FEEC2BF0CA
:1056D000200E366F003701370237033711EE33F0F3
:1056E0000A0E376FE7360A0EE75CD8B0E76EE55270
:1056F000372F72EF2BF0362F6AEF2BF034B1298160
:10570000D890120001010A0E346F200E366F11EE90
:1057100029F03451376F0A0ED890E652D8B0E726F8
:10572000E732372F8DEF2BF0033302330133003391
:10573000362F87EF2BF0E750FF0FD8A00335D8B0F6
:10574000120029B1CCEC2BF01200045100270551B6
:10575000D8B0053D01270651D8B0063D02270751B4
:10576000D8B0073D032712000051086F0151096F9F
:1057700002510A6F03510B6F12000101006B016BA4
:10578000026B036B12000101046B056B066B076B68
:1057900012000335D8A012000351800B001F011F17
:1057A000021F031F003FDCEF2BF0013FDCEF2BF06B
:1057B000023FDCEF2BF0032B342B032512000735BF
:1057C000D8A012000751800B041F051F061F071FDA
:1057D000043FF2EF2BF0053FF2EF2BF0063FF2EF24
:1057E0002BF0072B342B0725120000370137023727
:1057F0000337083709370A370B3712000101296BC5
:105800002A6B2B6B2C6B2D6B2E6B2F6B306B316BD4
:10581000326B336B120001012A510F0B2A6F2B518F
:105820000F0B2B6F2C510F0B2C6F2D510F0B2D6F5E
:105830002E510F0B2E6F2F510F0B2F6F30510F0B5F
:10584000306F31510F0B316F32510F0B326F3351BB
:105850000F0B336F120010A806D08994000EC76E8C
:10586000220EC66E05D08984000EC76E220EC66E4B
:10587000050EE82EFED7120010A802D0898401D0B0
:105880008994050EE82EFED712002BEC2CF09E9684
:10589000C69E000EC96EFF0E9EB602D0E82EFCD743
:1058A0009E96C69E000EC96EFF0E9EB602D0E82ED2
:1058B000FCD7C9CFAFF59E96C69E000EC96EFF0EEF
:1058C0009EB602D0E82EFCD7C9CFB0F59E96C69EF4
:1058D000000EC96EFF0E9EB602D0E82EFCD7C9CFCF
:1058E000B1F59E96C69E000EC96EFF0E9EB602D002
:1058F000E82EFCD7C9CFB2F59E96C69E000EC96EA3
:10590000FF0E9EB602D0E82EFCD7C9CFB3F59E9607
:10591000C69E000EC96EFF0E9EB602D0E82EFCD7C2
:10592000C9CFB4F59E96C69E000EC96EFF0E9EB6F8
:1059300002D0E82EFCD7C9CFB5F53CEC2CF0120014
:105940002BEC2CF09E96C69E800EC96EFF0E9EB666
:1059500002D0E82EFCD79E96C69EAFC5C9FFFF0EAB
:105960009EB602D0E82EFCD79E96C69EB0C5C9FF53
:10597000FF0E9EB602D0E82EFCD79E96C69EB1C5FD
:10598000C9FFFF0E9EB602D0E82EFCD79E96C69E9B
:10599000B2C5C9FFFF0E9EB602D0E82EFCD79E9678
:1059A000C69EB3C5C9FFFF0E9EB602D0E82EFCD737
:1059B0009E96C69EB4C5C9FFFF0E9EB602D0E82EC5
:1059C000FCD79E96C69EB5C5C9FFFF0E9EB602D0F7
:1059D000E82EFCD73CEC2CF012002BEC2CF09E9621
:1059E000C69E070EC96EFF0E9EB602D0E82EFCD7EB
:1059F0009E96C69E000EC96EFF0E9EB602D0E82E81
:105A0000FCD7C9CFAFF59E96C69E000EC96EFF0E9D
:105A10009EB602D0E82EFCD7C9CFB0F59E96C69EA2
:105A2000000EC96EFF0E9EB602D0E82EFCD7C9CF7D
:105A3000B1F59E96C69E000EC96EFF0E9EB602D0B0
:105A4000E82EFCD7C9CFB2F53CEC2CF02BEC2CF0B7
:105A50009E96C69E21C0C9FFFF0E9EB602D0E82EBC
:105A6000FCD79E96C69E000EC96EFF0E9EB602D053
:105A7000E82EFCD7C9CFB6F53CEC2CF012002BEC8D
:105A80002CF09E96C69E870EC96EFF0E9EB602D063
:105A9000E82EFCD79E96C69EAFC5C9FFFF0E9EB6E8
:105AA00002D0E82EFCD79E96C69EB0C5C9FFFF0E59
:105AB0009EB602D0E82EFCD79E96C69EB1C5C9FF01
:105AC000FF0E9EB602D0E82EFCD79E96C69EB2C5AB
:105AD000C9FFFF0E9EB602D0E82EFCD73CEC2CF09E
:105AE0002BEC2CF09E96C69E22C0C9FFFF0E9EB6E0
:105AF00002D0E82EFCD79E96C69EB6C5C9FFFF0E03
:105B00009EB602D0E82EFCD73CEC2CF012002BEC19
:105B10002CF09E96C69E870EC96EFF0E9EB602D0D2
:105B2000E82EFCD79E96C69E000EC96EFF0E9EB64E
:105B300002D0E82EFCD79E96C69E800EC96EFF0E40
:105B40009EB602D0E82EFCD79E96C69E800EC96EE9
:105B5000FF0E9EB602D0E82EFCD79E96C69E800E03
:105B6000C96EFF0E9EB602D0E82EFCD73CEC2CF09E
:105B700012002BEC2CF09E96C69E870EC96EFF0E6F
:105B80009EB602D0E82EFCD79E96C69E000EC96E29
:105B9000FF0E9EB602D0E82EFCD79E96C69E000E43
:105BA000C96EFF0E9EB602D0E82EFCD79E96C69E0A
:105BB000800EC96EFF0E9EB602D0E82EFCD79E96D0
:105BC000C69E800EC96EFF0E9EB602D0E82EFCD790
:105BD0003CEC2CF0120010A82DD02BEC2CF09E9653
:105BE000C69E22C0C9FFFF0E9EB602D0E82EFCD78B
:105BF0009E96C69E450EC96EFF0E9EB602D0E82E3A
:105C0000FCD73CEC2CF02BEC2CF09E96C69E8F0E15
:105C1000C96EFF0E9EB602D0E82EFCD79E96C69E99
:105C2000000EC96EFF0E9EB602D0E82EFCD73CECEB
:105C30002CF012002BEC2CF09E96C69E22C0C9FFC1
:105C4000FF0E9EB602D0E82EFCD79E96C69E010E91
:105C5000C96EFF0E9EB602D0E82EFCD73CEC2CF0AD
:105C60002BEC2CF09E96C69E910EC96EFF0E9EB632
:105C700002D0E82EFCD79E96C69EA50EC96EFF0EDA
:105C80009EB602D0E82EFCD73CEC2CF012002BEC98
:105C90002CF09E96C69E22C0C9FFFF0E9EB602D073
:105CA000E82EFCD79E96C69E810EC96EFF0E9EB64C
:105CB00002D0E82EFCD73CEC2CF012002BEC2CF0A0
:105CC0009E96C69E22C0C9FFFF0E9EB602D0E82E49
:105CD000FCD79E96C69E010EC96EFF0E9EB602D0E0
:105CE000E82EFCD73CEC2CF012002BEC2CF09E960E
:105CF000C69E910EC96EFF0E9EB602D0E82EFCD74E
:105D00009E96C69EA50EC96EFF0E9EB602D0E82EC8
:105D1000FCD73CEC2CF012002BEC2CF09E96C69E8F
:105D2000910EC96EFF0E9EB602D0E82EFCD79E964D
:105D3000C69E000EC96EFF0E9EB602D0E82EFCD79E
:105D40003CEC2CF012000501256B266B276B286BB1
:105D5000899A400EC76E200EC66E9E96C69E030E92
:105D6000C96EFF0E9EB602D0E82EFCD79E96C69E48
:105D700027C5C9FFFF0E9EB602D0E82EFCD79E961F
:105D8000C69E26C5C9FFFF0E9EB602D0E82EFCD7E0
:105D90009E96C69E25C5C9FFFF0E9EB602D0E82E70
:105DA000FCD79E96C69EC952FF0E9EB602D0E82E24
:105DB000FCD7898A0F01C950FF0A01E112000501D1
:105DC0002E51130A05E005012E51170A0CE01200AE
:105DD0000501F00E256FFF0E266F0F0E276F000EC8
:105DE000286FFCEF2EF00501F00E256FFF0E266FD9
:105DF000FF0E276F000E286F899A400EC76E200E87
:105E0000C66E9E96C69E030EC96EFF0E9EB602D04B
:105E1000E82EFCD79E96C69E27C5C9FFFF0E9EB6EC
:105E200002D0E82EFCD79E96C69E26C5C9FFFF0E5F
:105E30009EB602D0E82EFCD79E96C69E25C5C9FF09
:105E4000FF0E9EB602D0E82EFCD79E96C69EC95283
:105E5000FF0E9EB602D0E82EFCD7898A0F01C950EA
:105E6000FF0A1DE005012E51130A05E005012E5120
:105E7000170A0BE012000501000E256F000E266FB9
:105E8000100E276F000E286F12000501000E256FFF
:105E9000000E266F000E276F010E286F12000501FD
:105EA000256B266B276B286B05012E51130A05E025
:105EB00005012E51170A0CE012000501000E216F9A
:105EC000000E226F080E236F000E246F71EF2FF06B
:105ED0000501000E216F000E226F800E236F000E51
:105EE000246F21C500F122C501F123C502F124C5AB
:105EF00003F125C504F126C505F127C506F128C51E
:105F000007F133EC29F000C125F501C126F502C1E6
:105F100027F503C128F5899A400EC76E200EC66E7C
:105F20009E96C69E030EC96EFF0E9EB602D0E82E48
:105F3000FCD79E96C69E27C5C9FFFF0E9EB602D00F
:105F4000E82EFCD79E96C69E26C5C9FFFF0E9EB6BC
:105F500002D0E82EFCD79E96C69E25C5C9FFFF0E2F
:105F60009EB602D0E82EFCD79E96C69EC952FF0E62
:105F70009EB602D0E82EFCD7898AC950FF0A08E1F4
:105F800004C125F505C126F506C127F507C128F589
:105F9000D890050124332333223321332151F00BD0
:105FA000216F2167DBEF2FF02267DBEF2FF02367F4
:105FB000DBEF2FF0246771EF2FF00501100E25277E
:105FC000E86A2623E86A2723E86A28231200E86A99
:105FD00005012E51130A06E005012E51170A0BE0A8
:105FE000020E120005012851000A03E12751F00BAF
:105FF00007E0010E120005012851000A01E0010E20
:10600000120029C500F12AC501F12BC502F12CC5EA
:1060100003F125C504F126C505F127C506F128C5FC
:1060200007F1C2EC2AF003BF1200E7EC2FF0D8A46E
:1060300079EF30F0899A400EC76E200EC66E9E969C
:10604000C69E060EC96EFF0E9EB602D0E82EFCD785
:10605000898A899A9E96C69E020EC96EFF0E9EB6CA
:1060600002D0E82EFCD79E96C69E27C5C9FFFF0E1C
:106070009EB602D0E82EFCD79E96C69E26C5C9FFC6
:10608000FF0E9EB602D0E82EFCD79E96C69E25C572
:10609000C9FFFF0E9EB602D0E82EFCD79E96C69E84
:1060A000000EC96EFF0E9EB602D0E82EFCD7898A7C
:1060B000899A9E96C69E050EC96EFF0E9EB602D0A8
:1060C000E82EFCD79E96C69EC952FF0E9EB602D001
:1060D000E82EFCD7C9B062EF30F0898A0501100EB6
:1060E0002527E86A2623E86A2723E86A282301EFA0
:1060F00030F01200899A400EC76E200EC66E9E9632
:10610000C69E060EC96EFF0E9EB602D0E82EFCD7C4
:10611000898A899A9E96C69EC70EC96EFF0E9EB644
:1061200002D0E82EFCD7898A0501256B266B276BE8
:10613000286B1200899A400EC76E200EC66E9E967E
:10614000C69E050EC96EFF0E9EB602D0E82EFCD785
:106150009E96C69EC952FF0E9EB602D0E82EFCD770
:10616000C9CF37F5898A1200899A400EC76E200E72
:10617000C66E9E96C69EB90EC96EFF0E9EB602D022
:10618000E82EFCD7898A1200899A400EC76E200E2D
:10619000C66E9E96C69EAB0EC96EFF0E9EB602D010
:1061A000E82EFCD7898AFF0EE82EFED71200E7EC16
:1061B0002FF0D8A41200899A400EC76E200EC66E2A
:1061C0009E96C69E030EC96EFF0E9EB602D0E82EA6
:1061D000FCD79E96C69E27C5C9FFFF0E9EB602D06D
:1061E000E82EFCD79E96C69E26C5C9FFFF0E9EB61A
:1061F00002D0E82EFCD79E96C69E25C5C9FFFF0E8D
:106200009EB602D0E82EFCD79E96C69EC952FF0EBF
:106210009EB602D0E82EFCD7898A0F01C950FF0A2A
:10622000D8A4D2EF31F00501FE0E376F45EC2CF00B
:10623000AFC538F5B0C539F5B1C53AF5B2C53BF5CE
:10624000B3C53CF5B4C53DF5B5C53EF50784B6C14B
:1062500066F1B7C167F1B8C168F1B9C169F14BC165
:106260004FF14CC150F14DC151F14EC152F157C1E6
:1062700059F158C15AF1C6EC1FF000C13FF501C1F8
:1062800040F502C141F503C142F50501616750EFD8
:1062900031F0626750EF31F0636750EF31F06467BF
:1062A00054EF31F061EF31F061C504F162C505F1E1
:1062B00063C506F164C507F1C2EC2AF003BFD2EF53
:1062C00031F059C143F55AC144F5B9C545F5BAC5D0
:1062D00046F507940501110E326F899A400EC76E7C
:1062E000200EC66E9E96C69E060EC96EFF0E9EB608
:1062F00002D0E82EFCD7898A899A9E96C69E020E05
:10630000C96EFF0E9EB602D0E82EFCD79E96C69EA2
:1063100027C5C9FFFF0E9EB602D0E82EFCD79E9679
:10632000C69E26C5C9FFFF0E9EB602D0E82EFCD73A
:106330009E96C69E25C5C9FFFF0E9EB602D0E82ECA
:10634000FCD725EE37F0322F02D0B2EF31F09E9617
:10635000C69EDECFC9FFFF0E9EB602D0E82EFCD748
:10636000A3EF31F0898A899A9E96C69E050EC96E62
:10637000FF0E9EB602D0E82EFCD79E96C69EC9524E
:10638000FF0E9EB602D0E82EFCD7C9B0BDEF31F0AB
:10639000898A0501100E2527E86A2623E86A272343
:1063A000E86A2823120021C500F122C501F123C5A6
:1063B00002F124C503F1899A400EC76E200EC66E05
:1063C0009E96C69E0B0EC96EFF0E9EB602D0E82E9C
:1063D000FCD79E96C69E02C1C9FFFF0E9EB602D094
:1063E000E82EFCD79E96C69E01C1C9FFFF0E9EB641
:1063F00002D0E82EFCD79E96C69E00C1C9FFFF0EB4
:106400009EB602D0E82EFCD79E96C69EC952FF0EBD
:106410009EB602D0E82EFCD725EE37F00501100E0F
:10642000326F9E96C69EC952FF0E9EB602D0E82ECF
:10643000FCD7C9CFDEFF322F11EF32F0898A12006C
:10644000899A400EC76E200EC66E9E96C69E900E0E
:10645000C96EFF0E9EB602D0E82EFCD79E96C69E51
:10646000000EC96EFF0E9EB602D0E82EFCD79E9697
:10647000C69E000EC96EFF0E9EB602D0E82EFCD757
:106480009E96C69E000EC96EFF0E9EB602D0E82EE6
:10649000FCD79E96C69EC952FF0E9EB602D0E82E2D
:1064A000FCD7C9CF2DF59E96C69EC952FF0E9EB64B
:1064B00002D0E82EFCD7C9CF2EF5898A1200AEECA7
:1064C00029F0B9C5E8FFD70802E3AEEC29F0B9C559
:1064D000E8FFC80802E3AEEC29F0B9C5E8FFB90847
:1064E00002E3AEEC29F0B9C5E8FFAA0802E3AEEC7E
:1064F00029F0B9C5E8FF9B0802E3AEEC29F0EDEC0A
:106500002CF0B4EC30F0F29CF29E8B94C69AC290C0
:106510009482948C720ED36ED3A4FED789968A90FF
:106520009390FF0EE8CF00F0E82EFED7002EFCD7A8
:106530008150F294F29A9E909D909E929D92F29834
:0C654000F292F290F286F28E0300FF004F
:10BF0000E844F926000C160C2B0C3F0C520C640C68
:10BF1000760C860C960CA50CB30CC10CCF0CDC0C6B
:06BF2000E80CF40C000C1B
:0200000400F00A
:0100C800FE39
:00000001FF
